:100000000C945A280C9482280C9482280C948228F0
:100010000C9482280C9482280C9482280C948228B8
:100020000C9482280C9482280C9482280C948228A8
:100030000C9482280C9482280C9482280C94822898
:100040000C94F0310C9482280C94BE310C949831AD
:100050000C9482280C9482280C9482280C94822878
:100060000C9482280C9482280000000000000000FC
:100070000000000000000000000000000000000080
:10008000000000000000000000000C000C000C004C
:100090000C000C000C000C000C0000000C00000018
:1000A0000000000000000000000000001DC01DC096
:1000B00008800880088000000000000000000000A8
:1000C000000000000000000000000D800D800D8089
:1000D0000D803FC01B003FC01B001B001B001B000E
:1000E000000000000000000004001F80318031800B
:1000F00038001E000F000380318031803F00040073
:10010000040000000000000000001800240024008B
:1001100018C007801E0031800240024001800000AC
:100120000000000000000000000000000F001800A8
:10013000180018000C001D80370033001D800000DF
:1001400000000000000000000000000007000700A1
:100150000200020002000000000000000000000099
:100160000000000000000000000003000300060083
:100170000E000C000C000C000C000E00060003002A
:1001800003000000000000000000180018000C0030
:100190000600060006000600060006000C001C0013
:1001A00018000000000000000000060006003FC02C
:1001B0003FC00F001F8019800000000000000000F9
:1001C000000000000000000000000000000004002B
:1001D000040004003F80040004000400000000004C
:1001E000000000000000000000000000000000000F
:1001F00000000000000000000000060004000C00E9
:1002000008000800000000000000000000000000DE
:10021000000000003F80000000000000000000001F
:1002200000000000000000000000000000000000CE
:10023000000000000000000000000C000C000000A6
:10024000000000000000000000C000C0018001802C
:100250000300030006000C000C001800180030001A
:10026000300000000000000000000E001B00318084
:10027000318031803180318031801B000E000000E0
:100280000000000000000000000006003E00060024
:100290000600060006000600060006003FC000003B
:1002A000000000000000000000000F0019803180F5
:1002B0003180030006000C00180030003F80000071
:1002C000000000000000000000003F00618001808D
:1002D00003001F0003800180018061803F00000057
:1002E00000000000000000000000070007000F00F1
:1002F0000B001B00130033003F8003000F80000041
:10030000000000000000000000001F80180018001E
:1003100018001F0011800180018021801F00000053
:100320000000000000000000000007801C00180012
:100330003000370039803180318019800F00000093
:10034000000000000000000000007F0043000300E8
:1003500006000600060006000C000C000C00000061
:10036000000000000000000000001F00318031800C
:1003700031801F0031803180318031801F000000CA
:10038000000000000000000000001E00330031806B
:10039000318033801D800180030007003C00000095
:1003A000000000000000000000000000000000004D
:1003B0000C000C000000000000000C000C0000000D
:1003C000000000000000000000000000000000002D
:1003D0000300030000000000000006000400080005
:1003E00008000000000000000000000000C0030042
:1003F00004001800600018000400030000C00000A2
:1004000000000000000000000000000000000000EC
:1004100000007FC000007FC000000000000000005E
:100420000000000000000000000000006000180054
:100430000400030000C00300040018006000000076
:100440000000000000000000000000001F003180DC
:100450003180018007000C000C0000000C0000003F
:10046000000000000000000000000E00110021004C
:1004700021002700290029002700200011000E007C
:100480000000000000000000000000003F000F001E
:100490000900198019801F8030C030C079E0000049
:1004A0000000000000000000000000007F0031801C
:1004B000318031803F003180318031807F00000009
:1004C0000000000000000000000000001F4030C0DD
:1004D0006040600060006000604030801F000000ED
:1004E0000000000000000000000000007F003180DC
:1004F00030C030C030C030C030C031807F0000001C
:100500000000000000000000000000007F8030803C
:10051000308032003E003200308030807F8000002A
:100520000000000000000000000000007FC030401C
:10053000304032003E003200300030007C000000CD
:100540000000000000000000000000001E8031805C
:1005500060806000600067C0618031801F00000023
:100560000000000000000000000000007BC031809F
:10057000318031803F803180318031807BC000000C
:100580000000000000000000000000003FC0060066
:100590000600060006000600060006003FC0000038
:1005A0000000000000000000000000001FC0030069
:1005B0000300030003006300630063003E000000CB
:1005C0000000000000000000000000007BC031803F
:1005D000330036003C003E003300318079C000001B
:1005E0000000000000000000000000007E00180075
:1005F0001800180018001840184018407FC000006C
:10060000000000000000000000000000E0E060C00A
:1006100071C07BC06AC06EC064C060C0FBE00000F7
:1006200000000000000000000000000073C03180E6
:1006300039803D803580378033803180798000007B
:100640000000000000000000000000001F003180DA
:1006500060C060C060C060C060C031801F0000002A
:100660000000000000000000000000007F0031805A
:100670003180318031803F00300030007E0000004A
:100680000000000000000000000000001F0031809A
:1006900060C060C060C060C060C031801F000CC01E
:1006A0001F80000000000000000000007F0031807B
:1006B000318031803E003300318031807CE00000A9
:1006C0000000000000000000000000001F803180DA
:1006D000318038001F000380318031803F000000EE
:1006E0000000000000000000000000007F804C803F
:1006F0004C804C800C000C000C000C003F000000F3
:100700000000000000000000000000007BC03180FD
:100710003180318031803180318031801F00000094
:100720000000000000000000000000007BC03180DD
:1007300031801B001B001B000A000E000E00000091
:10074000000000000000000000000000FBE060C0AE
:1007500064C06EC06EC02A803B803B803180000048
:100760000000000000000000000000007BC031809D
:100770001B000E000E000E001B0031807BC000002D
:1007800000000000000000000000000079E030C020
:1007900019800F0006000600060006001F800000FA
:1007A0000000000000000000000000003F802180E9
:1007B0002300060004000C00188030803F800000F9
:1007C0000000000000000000000007800600060096
:1007D00006000600060006000600060006000600E9
:1007E00007800000000000003000300018001800F2
:1007F0000C000C000600030003000180018000C013
:1008000000C000000000000000001E0006000600FE
:1008100006000600060006000600060006000600A8
:100820001E0000000000000004000A000A00110081
:100830002080208000000000000000000000000078
:1008400000000000000000000000000000000000A8
:100850000000000000000000000000000000000098
:10086000000000000000FFE008000400020000009B
:100870000000000000000000000000000000000078
:100880000000000000000000000000000000000068
:100890001F00018001801F80318033801DC0000057
:1008A0000000000000000000000070003000300078
:1008B0003700398030C030C030C039807700000048
:1008C0000000000000000000000000000000000028
:1008D0001E80318060806000608031801F000000D9
:1008E0000000000000000000000003800180018083
:1008F0001D80338061806180618033801DC0000075
:1009000000000000000000000000000000000000E7
:100910001F00318060C07FC0600030C01F800000B9
:100920000000000000000000000007E00C000C00C8
:100930003F800C000C000C000C000C003F800000FD
:1009400000000000000000000000000000000000A7
:100950001DC0338061806180618033801D80018093
:1009600001801F0000000000000070003000300017
:100970003700398031803180318031807BC0000088
:10098000000000000000000000000600060000005B
:100990001E00060006000600060006003FC000001C
:1009A000000000000000000000000600060000003B
:1009B0003F000300030003000300030003000300E3
:1009C00003003E0000000000000070003000300016
:1009D000378036003C003C003600330077C0000012
:1009E000000000000000000000001E0006000600DD
:1009F0000600060006000600060006003FC00000D4
:100A000000000000000000000000000000000000E6
:100A10007F8036C036C036C036C036C076E00000B3
:100A200000000000000000000000000000000000C6
:100A30007700398031803180318031807BC0000087
:100A400000000000000000000000000000000000A6
:100A50001F00318060C060C060C031801F00000096
:100A60000000000000000000000000000000000086
:100A70007700398030C030C030C039803700300056
:100A800030007C00000000000000000000000000BA
:100A90001DC0338061806180618033801D80018052
:100AA000018007C0000000000000000000000000FE
:100AB0007B801CC018001800180018007F00000080
:100AC0000000000000000000000000000000000026
:100AD0001F8031803C001F00038031803F000000F8
:100AE00000000000000000000000180018001800BE
:100AF0007F00180018001800180018800F00000070
:100B000000000000000000000000000000000000E5
:100B10007380318031803180318033801DC000008E
:100B200000000000000000000000000000000000C5
:100B30007BC0318031801B001B000E000E000000C6
:100B400000000000000000000000000000000000A5
:100B5000F1E060C064C06EC03B803B80318000002B
:100B60000000000000000000000000000000000085
:100B70007BC01B000E000E000E001B007BC000009F
:100B80000000000000000000000000000000000065
:100B900079E030C0198019800B000F0006000600B4
:100BA0000C003E00000000000000000000000000FB
:100BB0003F80218003000E00180030803F8000003D
:100BC0000000000000000000000006000C000C0007
:100BD0000C000C000C0018000C000C000C000C00A9
:100BE00006000000000000000000060006000600ED
:100BF00006000600060006000600060006000600C5
:100C0000060000000000000000000C0006000600C6
:100C100006000600060003000600060006000600A7
:100C20000C000000000000000000000000000000B8
:100C300000001800248003000000000000000000F5
:100C40000000000000000000FFFFFFFFFFFFFFFFAC
:100C5000FFFFFFFFFFFFFFFFFFFC03FFFFFFFFFFA3
:100C6000FFFFFFFFFFFFFFFFFC02AAAAAAAAAAAA92
:100C7000AAAAAAAAFFFFFFFFFFFFFFFFFFFFFFFFD8
:100C8000FFFFFFFFFFFC03FFFFFFFFFFFFFFFFFF73
:100C9000FFFFFFFFFC02AAAAAAAAAAAAAAAAAAAAB6
:100CA000FFFFFFFFFFFFFFFFFFFFFFFFFFFFFFFF54
:100CB000FFFC03FFFFFFFFFFFFFFFFFFFFFFFFFF43
:100CC000FC02AAAAAAAAAAAAAAAAAAAAFFFFFFFF86
:100CD000FFFFFFFFFFFFFFFFFFFFFFFFFFFC03FF23
:100CE000FFFFFFFFFFFFFFFFFFFFFFFFFC02AAAABE
:100CF000AAAAAAAAAAAAAAAAFFFFFFFFFFFFFFFFAC
:100D0000FFFFFFFFFFFFFFFFFFFC03FFFFFFFFFFF2
:100D1000FFFFFFFFFFFFFFFFFC02AAAAAAAAAAAAE1
:100D2000AAAAAAAAFFFFFFFFFFFFFFFFFFFFFFFF27
:100D3000FFFFFFFFFFFC03FFFFFFFFFFFFFFFFFFC2
:100D4000FFFFFFFFFC02AAAAAAAAAAAAAAAAAAAA05
:100D5000FFFFFFFFFFFFFFFFFFFFFFFFFFFFFFFFA3
:100D6000FFFC03FFFFFFFFFFFFFFFFFFFFFFFFFF92
:100D7000FC02AAAAAAAAAAAAAAAAAAAAFFFFFFFFD5
:100D8000FFFFFFFFFFFFFFFFFFFFFFFFFFFC03FF72
:100D9000FFFFFFFFFFFFFFFFFFFFFFFFFC02AAAA0D
:100DA000AAAAAAAAAAAAAAAAFFFFFFFFFFFFFFFFFB
:100DB000FFFFFFFFFFFFFFFFFFFC03FFFFFFFFFF42
:100DC000FFFFFFFFFFFFFFFFFC02AAAAAAAAAAAA31
:100DD000AAAAAAAAFFFFFFFFFFFFFFFFFFFFFFFF77
:100DE000FFFFFFFFFFFC03FFFFFFFFFFFFFFFFFF12
:100DF000FFFFFFFFFC02AAAAAAAAAAAAAAAAAAAA55
:100E0000FFFFFFFFFFFFFFFFFFFFFFFFFFFFFFFFF2
:100E1000FFFC03FFD5555555555555555555555F4F
:100E2000FC02AAAAAAAAAAAAAAAAAAAAFFFFFFFF24
:100E3000FFFFFFFFFFFFFFFFFFFFFFFFFFFC03FFC1
:100E4000D5555555555555555555555FFC02AAAACA
:100E5000AAAAAAAAAAAAAAAAFFFFFFFFFFFFFFFF4A
:100E6000FFFFFFFFFFFFFFFFFFFC03FFD5555555B9
:100E7000555555555555555FFC02AAAAAAAAAAAAC6
:100E8000AAAAAAAAFFFFFFFFFFFFFFFFFFFFFFFFC6
:100E9000FFFFFFFFFFFC03FFD55555555555555531
:100EA0005555555FFC02AAAAAAAAAAAAAAAAAAAA42
:100EB000FFFFFFFFFFFFFFFFFFFFFC00FFFFFFFF44
:100EC000FFFC03FFD5555555555555555555555F9F
:100ED000FC02AAAAAAAAAAAAAAAAAAAAFFFFFFFF74
:100EE000FFFFFFFFFFFFC00003FFFFFFFFFC03FF4B
:100EF000D55FFFFFFFFFFFFFFFFFD55FFC02AAAA40
:100F0000AAAAAAAAAAAAAAAAFFFFFFFFFFFFFFFF99
:100F1000FFFC000000FFFFFFFFFC03FFD55FFFFFAA
:100F2000FFFFFFFFFFFFD55FFC02AAAAAAAAAAAA99
:100F3000AAAAAAAAFFFFFFFFFFFFFFFFFFF000A87A
:100F4000003FFFFFFFFC03FFD55FFFFFFFFFFFFF39
:100F5000FFFFD55FFC02AAAAAAAAAAAAAAAAAAAABD
:100F6000FFFFFFFFFFFFFFFFFFC00AAA800FFFFF89
:100F7000FFFC03FFD55FFFFFFFFFFFFFFFFFD55F14
:100F8000FC02AAAAAAAAAAAAAAAAAAAAFFFFFFFFC3
:100F9000FFFFFFFFFF002AAAA803FFFFFFFC03FFDC
:100FA000D55FFFFFFFFFFFFFFFFFD55FFC02AAAA8F
:100FB000AAAAAAAAAAAAAAAAFFFFFFFFFFFFFFFFE9
:100FC000F000AAAAAA03FFFFFFFC03FFD55FFFFF03
:100FD000F55555555557D55FFC02AAAAAAAAAAAA43
:100FE000AAAAAAAAFFFFFFFFFFFFFFFF0002AAAA0B
:100FF000AA03FFFFFFFC03FFD55F55555555555517
:101000005557D55FFC02AAAAAAAAAAAAAAAAAAAA5E
:10101000FFFFFFFFFFFFFFF00002AAAAAA00FFFFE9
:10102000FFFC03FFD55F5555555555555557D55FB1
:10103000FC02AAAAAAAAAAAAAAAAAAAAFFFFFFFF12
:10104000FFFFFF00000AAAAAAA00FFFFFFFC03FFA0
:10105000D55F5555555555555557D55FFC02AAAA2C
:10106000AAAAAAAAAAAAAAAAFFFFFFFFFFFFFF0037
:101070002AAAAAAAAA00FFFFFFFC03FFD55F5555C5
:10108000555555555557D55FFC02AAAAAAAAAAAA32
:10109000AAAAAAAAFFFFFFFFFFFFFC00AAAAAAAA0A
:1010A000AA00FFFFFFFC03FFD55F5557FFFFFFFFBF
:1010B000FFFFD55FFC02AAAAAAAAAAAAAAAAAAAA5C
:1010C000FFFFFFFFFFFFF00AAAAAAAAAAA00FFFFDC
:1010D000FFFC03FFD55F55555FFFFFFFFFFFD55FA7
:1010E000FC02AAAAAAAAAAAAAAAAAAAAFFFFFFFF62
:1010F000FFFFF02AAAAAAAAAAA00FFFFFFFC03FF8B
:10110000D55F5555557FFFFFFFFFD55FFC02AAAAAB
:10111000AAAAAAAAAAAAAAAAFFFFFFFFFFFFC02A9B
:10112000AAAAAAAAAA00FFFFFFFC03FFD55FFD55EC
:1011300055557FFFFFFFD55FFC02AAAAAAAAAAAA5B
:10114000AAAAAAAAFFFFFFFFFFFFC0AAAAAAAAAAEB
:10115000AA00FFFFFFFC03FFD55FFFFD555555FFBC
:10116000FFFFD55FFC02AAAAAAAAAAAAAAAAAAAAAB
:10117000FFFFFFFFFFFFC0AAAAAAAAAAAA00FFFFBB
:10118000FFFC03FFD55FFFFFFD55555FFFFFD55FF8
:10119000FC02AAAAAAAAAAAAAAAAAAAAFFFFFFFFB1
:1011A000FFFFC0AAAAAAAAAAAA00FFFFFFFC03FF8A
:1011B000D55FFFFFFFFD555FFFFFD55FFC02AAAAC9
:1011C000AAAAAAAAAAAAAAAAFFFFFFFFFFFFC0AA6B
:1011D000AAAAAAAAAA00FFFFFFFC03FFD55FFFFF90
:1011E000FD55555FFFFFD55FFC02AAAAAAAAAAAACD
:1011F000AAAAAAAAFFFFFFFFFFFFC0AAAAAAAAAA3B
:10120000AA00FFFFFFFC03FFD55FFFFD5555555FAB
:10121000FFFFD55FFC02AAAAAAAAAAAAAAAAAAAAFA
:10122000FFFFFFFFFFFFC0AAAAAAAAAAAA00FFFF0A
:10123000FFFC03FFD55FFD55555557FFFFFFD55FF9
:10124000FC02AAAAAAAAAAAAAAAAAAAAFFFFFFFF00
:10125000FFFFC02AAAAAAAAAAA00FFFFFFFC03FF59
:10126000D55F55555557FFFFFFFFD55FFC02AAAA72
:10127000AAAAAAAAAAAAAAAAFFFFFFFFFFFFC02A3A
:10128000AAAAAAAAAA00FFFFFFFC03FFD55F555533
:1012900057FFFFFFFFFFD55FFC02AAAAAAAAAAAACE
:1012A000AAAAAAAAFFFFFFFFFFFFF00AAAAAAAAAFA
:1012B000AA00FFFFFFFC03FFD55F5555FFFFFFFFAF
:1012C000FFFFD55FFC02AAAAAAAAAAAAAAAAAAAA4A
:1012D000FFFFFFFFFFC3F002AAAAAAAAAA00FFFF0E
:1012E000FFFC03FFD55F55555555555557FFD55F45
:1012F000FC02AAAAAAAAAAAAAAAAAAAAFFFFFFFF50
:10130000FFF0FC00AAAAAAAAAA00FFFFFFFC03FFA5
:10131000D55F5555555555555557D55FFC02AAAA69
:10132000AAAAAAAAAAAAAAAAFFFFFFFFFFF03F0043
:1013300002AAAAAAAA00FFFFFFFC03FFD55F55552A
:10134000555555555557D55FFC02AAAAAAAAAAAA6F
:10135000AAAAAAAAFFFFFFFFFFFC0FC002AAAAAA1F
:10136000AA00FFFFFFFC03FFD55F555555555555A6
:101370005557D55FFC02AAAAAAAAAAAAAAAAAAAAEB
:10138000FFFFFFFFFFFF0FFC02AAAAAAAA00FFFFB0
:10139000FFFC03FFD55FFFFFF55555555557D55F4A
:1013A000FC02AAAAAAAAAAAAAAAAAAAAFFFFFFFF9F
:1013B000FFFFCFFC02AAAAAAAA00FFFFFFFC03FFBF
:1013C000D55FFFFFFFFFFFFFFFFFD55FFC02AAAA6B
:1013D000AAAAAAAAAAAAAAAAFFFFFFFF0FFFCFFCE8
:1013E00002AAAAAAAA00FFFFFFFC03FFD55FFFFF26
:1013F000FFFFFFFFFFFFD55FFC02AAAAAAAAAAAAC5
:10140000AAAAAAAAFFFFFFFF00FF03FC02AAAAAA3A
:10141000AA00FFFFFFFC03FFD55FFFFFFFFFFFFFF9
:10142000FD57D55FFC02AAAAAAAAAAAAAAAAAAAA92
:10143000FFFFFFFFC00C00FC02AAAAAAAA00FFFF40
:10144000FFFC03FFD55FFFFFFFFFFFFF5557D55F91
:10145000FC02AAAAAAAAAAAAAAAAAAAAFFFFFFFFEE
:10146000FC0003FC02AAAAAAAA00FFFFFFFC03FFDC
:10147000D55FFFFFFFFFFF555557D55FFC02AAAAB6
:10148000AAAAAAAAAAAAAAAAFFFFFFFFFFF00FFF13
:1014900000AAAAAAAA00FFFFFFFC03FFD55FFFFF77
:1014A000FFFFD5555557D55FFC02AAAAAAAAAAAA3A
:1014B000AAAAAAAAFFFFFFFFFFF00FFF002AAAAA0D
:1014C000AA00FFFFFFFC03FFD55FFFFFFFD55555C7
:1014D0005557D55FFC02AAAAAAAAAAAAAAAAAAAA8A
:1014E000FFFFFFFFFFF03FFFC002AAAAAA00FFFF15
:1014F000FFFC03FFD55FFFFFF55555555557D55FE9
:10150000FC02AAAAAAAAAAAAAAAAAAAAFFFFFFFF3D
:10151000FFC03FFFF00000AAAA00FFFFFFFC03FF8F
:10152000D55FFFF555555555557FD55FFC02AAAAE5
:10153000AAAAAAAAAAAAAAAAFFFFFFF000003FFF30
:10154000FC0002AAAA00FFFFFFFC03FFD55FFD55C8
:10155000555555557FFFD55FFC02AAAAAAAAAAAA8B
:10156000AAAAAAAAFFFFFFF000003FFFFFF002AA0D
:10157000AA00FFFFFFFC03FFD55F55555555555594
:101580007FFFD55FFC02AAAAAAAAAAA80AAAAAAAA9
:10159000FFFFFFFFFFF03FFFFFFC02AAAA00FFFFD3
:1015A000FFFC03FFD55F555555557F557FFFD55F30
:1015B000FC02AAAAAAAAAAA002AAAAAAFFFFFFFF3F
:1015C000FFF00FFFFFFC02AAAA00FFFFFFFC03FFD2
:1015D000D55F5555557FFF557FFFD55FFC02AAAA01
:1015E000AAAAAAA002AAAAAAFFFFFFFFFFF003FF70
:1015F000FFFF02AAAA03FFFFFFFC03FFD55F5555BB
:101600007FFFFF557FFFD55FFC02AAAAAAAAAAA85E
:101610000AAAAAAAFFFFFFFFFFC000FFFFFF00AA60
:10162000A803FFFFFFFC03FFD55F557FFFFFFF55BA
:101630007FFFD55FFC02AAAAAAAAAAAAAAAAAAAA56
:10164000FFFFFFFFFF00000300FFC00AA003FFFF32
:10165000FFFC03FFD55F55557FFFFF557FFFD55F2B
:10166000FC02AAAAAAAAAAAAAAAAAAAAFFFFFFFFDC
:10167000F00FC000003FC000000FFFFFFFFC03FFA2
:10168000D55F555555FFFF557FFFD55FFC02AAAAD0
:10169000AAAAAAAAAAAAAAAAFFFFFFFFC0FFF0004F
:1016A000000FF000003FFFFFFFFC03FFD55F555523
:1016B0005555FF557FFFD55FFC02AAAAAAAAAAAA80
:1016C000AAAAAAAAFFFFFFFFC3FFF00003C3FF00FF
:1016D00003FFFFFFFFFC03FFD55FD5555555575559
:1016E0007FFFD55FFC02AAAAAAAAAAAAAAAAAAAAA6
:1016F000FFFFFFFFFFFFC3FC3FF0FFF03FFFFFFFD7
:10170000FFFC03FFD55FFF55555555557FFFD55F4E
:10171000FC02AAAAAAAAAAAAAAAAAAAAFFFFFFFF2B
:10172000FFFFC3FF3FF03FFFFFFFFFFFFFFC03FF93
:10173000D55FFFFD555555555FFFD55FFC02AAAA41
:10174000AAAAAAAAAAAAAAAAFFFFFFFFFFFF0FFF41
:101750003FFC3FFFFFFFFFFFFFFC03FFD55FFFFFE5
:10176000FD555555555FD55FFC02AAAAAAAAAAAA9B
:10177000AAAAAAAAFFFFFFFFFFFF0FFF3FFF0FFF6D
:10178000FFFFFFFFFFFC03FFD55FFFFFFFF5555590
:101790005557D55FFC02AAAA0000000002AAAAAA17
:1017A000FFFFFFFFFFFC3FFF0FFFCFFFFFFFFFFF2C
:1017B000FFFC03FFD55FFFFFFFFFF5555557D55FD2
:1017C000FC02AAAA0000000002AAAAAAFFFFFFFFCB
:1017D000FFFFFFFF0FFFFFFFFFFFFFFFFFFC03FF08
:1017E000D55FFFFFFFFFFFD55557D55FFC02AAAAC3
:1017F000AA80AAA02AAAAAAAFFFFFFFFFFFFFFFF55
:101800000FFFFFFFFFFFFFFFFFFC03FFD55FFFFFA1
:10181000FFFFFFFF5557D55FFC02AAAAAA82AAA81C
:101820000AAAAAAAFFFFFFFFFFFFFFFFFFFFFFFFBC
:10183000FFFFFFFFFFFC03FFD55FFFFFFFFFFFFF81
:10184000FF57D55FFC02AAAAAA82AAAA0AAAAAAA34
:10185000FFFFFFFFFFFFFFFFFFFFFFFFFFFFFFFF98
:10186000FFFC03FFD55FFFFFFFFFFFFFFFFFD55F1B
:10187000FC02AAAAAA82AAAA82AAAAAAFFFFFFFF1A
:10188000FFFFFFFFFFFFFFFFFFFFFFFFFFFC03FF67
:10189000D55FFFFFFFFFFFFFFFFFD55FFC02AAAA96
:1018A000AA82AAAA82AAAAAAFFFFFFFFFFFFFFFF40
:1018B000FFFFFFFFFFFFFFFFFFFC03FFD55FFFFF01
:1018C000FFFFFFFFFFFFD55FFC02AAAAAAA0AAAAFA
:1018D00082AAAAAAFFFFFFFFFFFFFFFFFFFFFFFF94
:1018E000FFFFFFFFFFFC03FFD55FFFFFFFFFFFFFD1
:1018F000FFFFD55FFC02AAAAAAA02AAA02AAAAAA46
:10190000FFFFFFFFFFFFFFFFFFFFFFFFFFFFFFFFE7
:10191000FFFC03FFD5555555555555555555555F44
:10192000FC02AAAAAAA800000AAAAAAAFFFFFFFF0F
:10193000FFFFFFFFFFFFFFFFFFFFFFFFFFFC03FFB6
:10194000D5555555555555555555555FFC02AAAABF
:10195000AAAA00002AAAAAAAFFFFFFFFFFFFFFFF13
:10196000FFFFFFFFFFFFFFFFFFFC03FFD5555555AE
:10197000555555555555555FFC02AAAAAAAAAAAABB
:10198000AAAAAAAAFFFFFFFFFFFFFFFFFFFFFFFFBB
:10199000FFFFFFFFFFFC03FFD55555555555555526
:1019A0005555555FFC02AAAAAAAAAAAAAAAAAAAA37
:1019B000FFFFFFFFFFFFFFFFFFFFFFFFFFFFFFFF37
:1019C000FFFC03FFD5555555555555555555555F94
:1019D000FC02AAAAAAAAAAAAAAAAAAAAFFFFFFFF69
:1019E000FFFFFFFFFFFFFFFFFFFFFFFFFFFC03FF06
:1019F000FFFFFFFFFFFFFFFFFFFFFFFFFC02AAAAA1
:101A0000AAAAAAAAAAAAAAAA000000000000000086
:101A10000000000000000000000003FFFFFFFFFFC8
:101A2000FFFFFFFFFFFFFFFFFC02AAAAAAAA002AEE
:101A3000AAAAAAAA000000000000000000000000FE
:101A400000000000000003FFFFFFFFFFFFFFFFFF9C
:101A5000FFFFFFFFFC02AAAAAAA8002A8AAAAAAA34
:101A60000000000000000000000000000000000076
:101A7000000003FFFFFFFFFFFFFFFFFFFFFFFFFF70
:101A8000FC02AAAAAAA0282A82AAAAAA00000000E8
:101A9000000000000000000000000000000003FF44
:101AA000FFFFFFFFFFFFFFFFFFFFFFFFFC02AAAAF0
:101AB000AA80A82A82AAAAAAFFFFFFFFFFFFFFFFB2
:101AC000FFFFFFFFFFFFFFFFFFFC03FFFFFFFFFF25
:101AD000FFFFFFFFFFFFFFFFFC02AAAAAA82A82ABE
:101AE00082AAAAAAFFFFFFFFFFFFFFFFFFFFFFFF82
:101AF000FFFFFFFFFFFC03FFFFFFFFFFFFFFFFFFF5
:101B0000FFFFFFFFFC02AAAAAA82A82A82AAAAAA09
:101B1000FFFFFFFFFFFFFFFFFFFFFFFFFFFFFFFFD5
:101B2000FFFC03FFFFFFFFFFFFFFFFFFFFFFFFFFC4
:101B3000FC02AAAAAA82A82A82AAAAAAFFFFFFFFD9
:101B4000FFFFFFFFFFFFFFFFFFFFFFFFFFFC03FFA4
:101B5000FFFFFFFFFFFFFFFFFFFFFFFFFC02AAAA3F
:101B6000AA82A82A02AAAAAAFFFFFFFFFFFFFFFF7F
:101B7000FFFFFFFFFFFFFFFFFFFC03FFFFFFFFFF74
:101B8000FFFFFFFFFFFFFFFFFC02AAAAAAA0A82AEF
:101B90000AAAAAAAFFFFFFC0000FFFFFFFFFFFFF77
:101BA000FFFFFFFFFFFC03FFFFFFFFFFFFFFFFFF44
:101BB000FFFFFFFFFC02AAAAAAA000000AAAAAAA85
:101BC000FFFFFF000003FFFFFFFFFFFFFFFFFFFF1F
:101BD000FFFC03FFFFFFFFFFFFFFFFFFFFFFFFFF14
:101BE000FC02AAAAAAA800002AAAAAAAFFFFF00338
:101BF000FC000FFFFFFFFFFFFFFFFFFFFFFC03FFE6
:101C0000FFFFFFFFFFFFFFFFFFFFFFFFFC02AAAA8E
:101C1000AAAA8002AAAAAAAAFFFF00FFFFFC03FF4C
:101C2000FFFFFFFFFFFFFFFFFFFC03FFFFFFFFFFC3
:101C3000FFFFFFFFFFFFFFFFFC02AAAAAAAAAAAAB2
:101C4000AAAAAAAAFFFC0FFFFFFF003FFFFFFFFFAA
:101C5000FFFFFFFFFFFC03FFFFFFFFFFFFFFFFFF93
:101C6000FFFFFFFFFC02AAAAAAAAAAAAAAAAAAAAD6
:101C7000FFF00FC03C0FC00FFFFFFFFFFFFFFFFF94
:101C8000FFFC03FFFFFFFFFFFFFFFFFFFFFFFFFF63
:101C9000FC02AAAA800002AAAAAAAAAAFFC03F0020
:101CA0000F03F003FFFFFFFFFFFFFFFFFFFC03FF3A
:101CB000FFFFFFFFFFFFFFFFFFFFFFFFFC02AAAADE
:101CC0008000000002AAAAAAFF003C000F00F00357
:101CD000FFFFFFFFFFFFFFFFFFFC03FFFFFFFFF022
:101CE0000000000FFFFFFFFFFC02AAAAAAAAAAA0F9
:101CF00002AAAAAAFC003C000F003000FFFFFFFF71
:101D0000FFFFFFFFFFFC03FFFFFFF00000000000EC
:101D10003FFFFFFFFC02AAAAAAAAAAA802AAAAAA8F
:101D2000FC003C000F003C0000000000000000032D
:101D3000FFFC03FFFFFF00000000000003FFFFFFA8
:101D4000FC02AAAAAAAAAA002AAAAAAAF0003F00EC
:101D50000F003C000000000000000003FFFC03FF38
:101D6000FFFC000000000000003FFFFFFC02AAAAE9
:101D7000AAAA800AAAAAAAAAF0000F003F003C0063
:101D80000000000000000003FFFC03FFFFF0000064
:101D900000000000000FFFFFFC02AAAAAAA802AAE6
:101DA000AAAAAAAAC0000FFFFC003C000000000085
:101DB00000000003FFFC03FFFFC000000FFFFFF067
:101DC0000003FFFFFC02AAAAAAA800AAAAAAAAAA1C
:101DD000C00003FFF000000000000000000000034E
:101DE000FFFC03FFFF0003C003FFFFFFC000FFFF76
:101DF000FC02AAAAAAAAA002AAAAAAAAC000000F24
:101E0000000000000000000000000003FFFC03FFD2
:101E1000FC003FF000FFFFFFFC00FFFFFC02AAAA4E
:101E2000AAAAAA800AAAAAAAC0000000000000006C
:101E300002AAAAAAAA000003FFFC03FFFC00FFFC01
:101E4000003FFFFFFF003FFFFC02AAAAAAAAAAAA1E
:101E500002AAAAAAC00000000000000002AAAAAAC2
:101E6000A8000003FFFC03FFFC03FFFF003FFFFF90
:101E7000FFC03FFFFC02AAAAA800000002AAAAAA6B
:101E8000C00000000000000002AAAAAAA0000003EF
:101E9000FFFC03FFF003FFFF000FFFFFFFC03FFF4A
:101EA000FC02AAAA8000000002AAAAAAC000003F61
:101EB000FFF0000002AAAAAA80000003FFFC03FFB3
:101EC000F00FFFFFC003FFFFFFF00FFFFC02AAAA05
:101ED000800AAAAAAAAAAAAAC00003FFFFFF0000BC
:101EE00002AAAAAA00000003FFFC03FFF00FFFFFF5
:101EF000F000FFFFFFF00FFFFC02AAAAAAAAAAAAFD
:101F0000AAAAAAAAC0000FF03C3FC00002AAAAA831
:101F100000008003FFFC03FFF00FFFFFFC00FFFF4A
:101F2000FFF00FFFFC02AAAAAAAAAAAAAAAAAAAA12
:101F3000C0000F000C03F00002AAAAA00002800358
:101F4000FFFC03FFF00FFFFFFC003FFFFFF00FFF60
:101F5000FC02AAAAAAAAAAAAAAAAAAAAF0003C00B3
:101F60000F00F0000AAAAA80000A8003FFFC03FF0A
:101F7000F00FFFFFFF000FFFFFF00FFFFC02AAAA08
:101F8000AAAAAAAAAAAAAAAAF0003C000F00F000D6
:101F90002AAAAA0000AA8003FFFC03FFFC03FFFF9C
:101FA000FFC00FFFFFC00FFFFC02AAAAAAAAAAAA9D
:101FB000AAAAAAAAF0003C000F003C002AAAA80086
:101FC00002AA8003FFFC03FFFC03FFFFFFF003FFF7
:101FD000FFC03FFFFC02AAAAAAAAAAAAAAAAAAAA62
:101FE000FC003C000F003C00AAAAA0000AAA800343
:101FF000FFFC03FFFC00FFFFFFF000FFFF003FFFBF
:10200000FC02AAAAAAAAAAAAAAAAAAAAFC000F0023
:102010003F003C00AAAA80002AAA8003FFFC03FF1D
:10202000FF003FFFFFFC003FF0003FFFFC02AAAAB9
:10203000AAAAAAAAAAAAAAAAFF000FC0FC003C0248
:10204000AAA80000AAAA8003FFFC03FFFF0003FF69
:10205000FFFF003FC000FFFFFC02AAAAAAAAAAAA8B
:10206000AAAAAAAAFFC003FFFC003C02AAA0000281
:10207000AAAA8003FFFC03FFFFC0000FFFFF0000C0
:102080000003FFFFFC02AAAAAAAAAAAAAAAAAAAAAD
:10209000FFF000FFC0000000AA80000AAAAA800387
:1020A000FFFC03FFFFF00000000000000003FFFF43
:1020B000FC02AAAAAAAAAAAAAAAAAAAAFFFC000083
:1020C000000000002A00002AAAAA8003FFFC03FFE8
:1020D000FFFC000000000000003FFFFFFC02AAAA76
:1020E000AAAAAAAAAAAAAAAAFFFF000000000000A2
:1020F000080000AAAAAA8003FFFC03FFFFFFC0009C
:102100000000000000FFFFFFFC02AAAAAAAAAAAAD8
:10211000AAAAAAAAFFFFC00000002800000002AA85
:10212000AAAA8003FFFC03FFFFFFFC0000000000E1
:102130000FFFFFFFFC02AAAAAAAAAAAAAAAAAAAAF1
:10214000FFFFC0000002AA0000000AAAAAAA80039A
:10215000FFFC03FFFFFFFFF00000000FFFFFFFFF8A
:10216000FC02AAAAAAAAAAAAAAAAAAAAFFFFC0020D
:10217000AAAAAA800000AAAAAAAA8003FFFC03FFB9
:10218000FFFFFFFFFFFFFFFFFFFFFFFFFC02AAAA09
:10219000AAAAAAAAAAAAAAAAFFFFC002AAAAAAA091
:1021A0000002AAAAAAAA8003FFFC03FFFFFFFFFF09
:1021B000FFFFFFFFFFFFFFFFFC02AAAAAAAAAAAA2D
:1021C000AAAAAAAAFFFFC002AAAAAAA80002AAAAAB
:1021D000AAAA8003FFFC03FFFFFFFFFFFFFFFFFF33
:1021E000FFFFFFFFFC02AAAAAAAAAAAAAAAAAAAA51
:1021F000FFFFC002AAAAAAA80002AAAAAAAA80034C
:10220000FFFC03FFFFFFFFFFFFFFFFFFFFFFFFFFDD
:10221000FC02AAAAAAAAA000AAAAAAAAFFFFC00210
:10222000AAAAAAAA0000AAAAAAAA8003FFFC03FFDE
:10223000FFFFFFFFFFFFFFFFFFFFFFFFFC02AAAA58
:1022400082AA80000AAAAAAAFFFFC002AAAAAAAA72
:1022500080002AAAAAAA8003FFFC03FFFFFFFFFF5A
:10226000FFFFFFFFFFFFFFFFFC02AAAA82AA82A8CE
:102270000AAAAAAAFFFFC002AAAAAAAAA0000AAA9A
:10228000AAAA8003FFFC03FFFFFFFFF00000000F7E
:10229000FFFFFFFFFC02AAAA82AA0AAA02AAAAAA10
:1022A000FFFFC002AAAAAAAAA80002AAAAAA80039B
:1022B000FFFC03FFFFFFF000000000003FFFFFFFF7
:1022C000FC02AAAA82AA0AAA82AAAAAAFFFFC0029C
:1022D000AAAAAAAAAA0000AAAAAA8003FFFC03FF2E
:1022E000FFFF00000000000003FFFFFFFC02AAAA9E
:1022F00082AA0AAA82AAAAAAFFFFC002AAAAAAAA16
:10230000AA8000AAAAAA8003FFFC03FFFFFC00002A
:1023100000000000003FFFFFFC02AAAAA0AA0AAA30
:1023200082AAAAAAFFFFC002AAAAAAAAAAA0002A51
:10233000AAAA8003FFFC03FFFFF0000000000000DA
:10234000000FFFFFFC02AAAAA0AA0AAA82AAAAAAB0
:10235000FFFFC002AAAAAAAAAAA8000AAAAA8003E2
:10236000FFFC03FFFFC000000FFFFFF00003FFFFB3
:10237000FC02AAAAA80A82AA0AAAAAAAFFFFC00265
:10238000AAAAAAAAAAA8000AAAAA8003FFFC03FF75
:10239000FF0003C003FFFFFFC000FFFFFC02AAAA6B
:1023A000AA0000000AAAAAAAFFFFC002AAAAAAAA13
:1023B000AAA0000AAAAA8003FFFC03FFFC003FF0CA
:1023C00000FFFFFFFC00FFFFFC02AAAAAA8000009A
:1023D0002AAAAAAAFFFFC002AAAAAAAAAA80002A19
:1023E000AAAA8003FFFC03FFFC00FFFC003FFFFFE5
:1023F000FF003FFFFC02AAAAAAAA000AAAAAAAAA48
:10240000FFFFC002AAAAAAAAAA0000AAAAAA800339
:10241000FFFC03FFFC03FFFF003FFFFFFFC03FFF88
:10242000FC02AAAAAAAAAAAAAAAAAAAAFFFFC0024A
:10243000AAAAAAAAA80002AAAAAA8003FFFC03FFCC
:10244000F003FFFF000FFFFFFFC03FFFFC02AAAA3F
:10245000AAAAAAAAAAAAAAAAFFFFC002AAAAAAAAC4
:10246000A0000AAAAAAA8003FFFC03FFF00FFFFF47
:10247000C003FFFFFFF00FFFFC02AAAAAAAAAAAAA4
:10248000AAAAAAAAFFFFC002AAAAAAAAA0002AAAC8
:10249000AAAA8003FFFC03FFF00FFFFFF000FFFF7D
:1024A000FFF00FFFFC02AAAAAAAAAAAA82AAAAAAB5
:1024B000FFFFC002AAAAAAAA8000AAAAAAAA800309
:1024C000FFFC03FFF00FFFFFFC00FFFFFFF00FFF1B
:1024D000FC02AAAAAAAAAAAA82AAAAAAFFFFC002C2
:1024E000AAAAAAAA0002AAAAAAAA8003FFFC03FF1A
:1024F000F00FFFFFFC003FFFFFF00FFFFC02AAAA56
:10250000AAAAAAAA82AAAAAAFFFFC002AAAAAAA83D
:102510000002AAAAAAAA8003FFFC03FFF00FFFFF94
:10252000FF000FFFFFF00FFFFC02AAAAAAAAAAAAA7
:1025300082AAAAAAFFFFC002AAAAAAA00002AAAA67
:10254000AAAA8003FFFC03FFFC03FFFFFFC00FFFED
:10255000FFC00FFFFC02AAAA8000000002AAAAAADC
:10256000FFFFC002AAAAAA800000AAAAAAAA800302
:10257000FFFC03FFFC03FFFFFFF003FFFFC03FFF73
:10258000FC02AAAA8000000002AAAAAAFFFFC002B9
:10259000AAAAAA0000002AAAAAAA8003FFFC03FF95
:1025A000FC00FFFFFFF000FFFF003FFFFC02AAAAB4
:1025B0008000000002AAAAAAFFFFC002AAAAA800DF
:1025C00000000AAAAAAA8003FFFC03FFFF003FFF46
:1025D000FFFC003FF0003FFFFC02AAAAA2AAAAAAA1
:1025E00082AAAAAAFFFFC002AAAAA800000002AA03
:1025F000AAAA8003FFFC03FFFF0003FFFFFF003FC9
:10260000C000FFFFFC02AAAAA0AAAAAA82AAAAAA9C
:10261000FFFFC002AAAAA0002A0000AAAAAA80035B
:10262000FFFC03FFFFC0000FFFFF00000003FFFFE0
:10263000FC02AAAAA82AAAAA82AAAAAAFFFFC002E2
:10264000AAAA8000AA80002AAAAA8003FFFC03FF8E
:10265000FFF00000000000000003FFFFFC02AAAA38
:10266000A82AAAAA82AAAAAAFFFFC002AAAA0002AE
:10267000AAA00002AAAA8003FFFC03FFFFFC00003F
:1026800000000000003FFFFFFC02AAAAAA2AAAAA93
:1026900082AAAAAAFFFFC002AAA80002AAA8000054
:1026A000AAAA8003FFFC03FFFFFFC0000000000098
:1026B00000FFFFFFFC02AAAAAAAAAAAAAAAAAAAA7B
:1026C000FFFFC002AAA0000AAAAA00002AAA80034B
:1026D000FFFC03FFFFFFFC00000000000FFFFFFFF7
:1026E000FC02AAAAAAAAAAAAAAAAAAAAFFFFC00288
:1026F000AA80002AAAAA80000AAA8003FFFC03FF7E
:10270000FFFFFFF00000000FFFFFFFFFFC02AAAA7F
:10271000AAAAAAAAAAAAAAAAFFFFC002AA0000AA55
:10272000AAAAA00002AA8003FFFC03FFFFFFFFFF8D
:10273000FFFFFFFFFFFFFFFFFC02AAAAAAAAAAAAA7
:10274000AAAAAAAAFFFFC002A80002AAAAAAA800D1
:1027500000AA8003FFFC03FFFFFFFFFFFFFFFFFF57
:10276000FFFFFFFFFC02AAAAAAAAAAAAAAAAAAAACB
:10277000FFFFC002A8000AAAAAAAAA00002A800392
:10278000FFFC03FFFFFFFFFFFFFFFFFFFFFFFFFF58
:10279000FC02AAAAAAAAAAAAAAAAAAAAFFFFC002D7
:1027A000A0002AAAAAAAAAA0000A8003FFFC03FF8D
:1027B000FFFFFFFFFFFFFFFFFFFFFFFFFC02AAAAD3
:1027C000AAAAAAAAAAAAAAAAFFFFC0028000AAAA25
:1027D000AAAAAAA800028003FFFC03FFFFFFFFFFD5
:1027E000FFFFFFFFFFFFFFFFFC02AAAAAAAAAAAAF7
:1027F000AAAAAAAAFFFFC0020000AAAAAAAAAAAA75
:1028000000008003FFFC03FFFFFFFFFFFFFFFFFF50
:10281000FFFFFFFFFC02AAAAAAAAAAAAAAAAAAAA1A
:10282000FFFFC0000002AAAAAAAAAAAA8000000369
:10283000FFFC03FFFFFFFFFFFFFFFFFFFFFFFFFFA7
:10284000FC02AAAAAAAAAAAAAAAAAAAAFFFFC00028
:10285000000AAAAAAAAAAAAAA0000003FFFC03FFD2
:10286000FFFFFFFFFFFFFFFFFFFFFFFFFC02AAAA22
:10287000AAAAAAAAAAAAAAAAFFFFC000002AAAAACC
:10288000AAAAAAAAA8000003FFFC03FFFFFFFFFFFC
:10289000FFFFFFFFFFFFFFFFFC02AAAAAAAAAAAA46
:1028A000AAAAAAAAFFFFC00000AAAAAAAAAAAAAA1C
:1028B000AA000003FFFC03FFFFFFFFFFFFFFFFFF76
:1028C000FFFFFFFFFC02AAAAAAAAAAAAAAAAAAAA6A
:1028D000FFFFC00000AAAAAAAAAAAAAAAA000003E7
:1028E000FFFC03FFFFFFFFFFFFFFFFFFFFFFFFFFF7
:1028F000FC02AAAAAAAAAAAAAAAAAAAAFFFFC00078
:10290000000000000000000000000003FFFC03FFC7
:10291000FFFFFFFFFFFFFFFFFFFFFFFFFC02AAAA71
:10292000AAAAAAAAAAAAAAAAFFFFC0000000000099
:102930000000000000000003FFFC03FFFFFFFFFF9B
:10294000FFFFFFFFFFFFFFFFFC02AAAAAAAAAAAA95
:10295000AAAAAAAAFFFFC000000000000000000011
:1029600000000003FFFC03FFFFFFFFFFFFFFFFFF6F
:10297000FFFFFFFFFC02AAAAAAAAAAAAAAAAAAAAB9
:10298000FFFFC00000000000000000000000000386
:10299000FFFC03FFFFFFFFFFFFFFFFFFFFFFFFFF46
:1029A000FC02AAAAAAAAAAAAAAAAAAAAFFFFC000C7
:1029B000000000000000000000000003FFFC03FF17
:1029C000FFFFFFF03FFFFFFFFF03FFFFFC02AAAA8C
:1029D000AA82AAAAA82AAAAAFFFFFFFFFFFFFFFF59
:1029E000FFFFFFFFFFFFFFFFFFFC03FFFFFFFF00F5
:1029F00003FFFFFFF0003FFFFC02AAAAAA82AAAAD7
:102A0000A00AAAAAFFFFFFFFFFFFFFFFFFFFFFFFD4
:102A1000FFFFFFFFFFFC03FFFFFFFF0003FFFFFFC0
:102A2000F0003FFFFC02AAAAAA8000AA8002AAAA7C
:102A3000FFFFFFFFFFFFFFFFFFFFFFFFFFFFFFFFA6
:102A4000FFFC03FFFFFFFC0000FFFFFFC0000FFFC4
:102A5000FC02AAAAAA80002A8282AAAAFFFFFFFF7C
:102A6000FFFFFFFFFFFFFFFFFFFFFFFFFFFC03FF75
:102A7000FFFFFC0000FFFFFFC0000FFFFC02AAAA3F
:102A8000AA80A82A82A0AAAAFFFFFFFFFFFFFFFFDC
:102A9000FFFFFFFFFFFFFFFFFFFC03FFFFFFFC0047
:102AA00000FFFFFFC0000FFFFC02AAAAAA82AA0A29
:102AB00082A0AAAAFFFFFFFFFFFFFFFFFFFFFFFFAC
:102AC000FFFFFFFFFFFC03FFFFFFFF0003FFFFFF10
:102AD000F0003FFFFC02AAAAAA82AA0A82A0AAAA20
:102AE000FFFFFFFFFFFFFFFFFFFFFFFFFFFFFFFFF6
:102AF000FFFC03FFFFFFFF0003FFFFFFF0003FFFAE
:102B0000FC02AAAAAA82AA0A82A0AAAAFFFFFFFF21
:102B1000FFFFFFFFFFFFFFFFFFFFFFFFFFFC03FFC4
:102B2000FFFFFFF03FFFFFFFFF03FFFFFC02AAAA2A
:102B3000AA82AA0A82A0AAAAFFFFFFFFFFFFFFFF47
:102B4000FFFFFFFFFFFFFFFFFFFC03FFFFFFFFFF94
:102B5000FFFFFFFFFFFFFFFFFC02AAAAAAA0A82A0F
:102B600082A0AAAAFFFFFFFFFFFFFFFFFFFFFFFFFB
:102B7000FFFFFFFFFFFC03FFFFFFFFFFFFFFFFFF64
:102B8000FFFFFFFFFC02AAAAAAA000000082AAAAD7
:102B9000FFFFFFFFFFFFFFFFFFFFFFFFFFFFFFFF45
:102BA000FFFC03FFFFFFFFFFFFFFFFFFFFFFFFFF34
:102BB000FC02AAAAAAA800800002AAAAFFFFFFFF9F
:102BC000FFFFFFFFFFFFFFFFFFFFFFFFFFFC03FF14
:102BD000FFFFFFFFFFFFFFFFFFFFFFFFFC02AAAAAF
:102BE000AAAAAAA02802AAAAFFFFFFFFFFFFFFFFD1
:102BF000FFFFFFFFFFFFFFFFFFFC03FFFFFFFFFFE4
:102C0000FFFFFFFFFFFFFFFFFC02AAAAAAAAAAAAD2
:102C1000AAAAAAAAFFFFFFFFFFFFFFFFFFFFFFFF18
:102C2000FFFFFFFFFFFC03FFFFFFFFFFFFFFFFFFB3
:102C3000FFFFFFFFFC02AAAAAAAAAAAAAAAAAAAAF6
:102C40000000000000000000000000000000000084
:102C5000000003FFFFFFFFFFFFFFFFFFFFFFFFFF7E
:102C6000FC02AAAAAAAAAAAAAAAAAAAA00000000C2
:102C7000000000000000000000000000000003FF52
:102C8000FFFFFFFFFFFFFFFFFFFFFFFFFC02AAAAFE
:102C9000AAAAAAAAAAAAAAAA0000000000000000E4
:102CA0000000000000000000000003FFFFFFFFFF26
:102CB000FFFFFFFFFFFFFFFFFC02AAAAAA800000A0
:102CC00002AAAAAA00000000000000000000000004
:102CD00000000000000003FFFFFFFFFFFFFFFFFFFA
:102CE000FFFFFFFFFC02AAAAAA80000002AAAAAA6C
:102CF000FFFFFFFFFFFFFFFFFFFFFFFFFFFFFFFFE4
:102D0000FFFC03FFFFFFFFFFFFFFFFFFFFFFFFFFD2
:102D1000FC02AAAAAAAAAAA82AAAAAAAFFFFFFFF97
:102D2000FFFFFFFFFFFFFFFFFFFFFFFFFFFC03FFB2
:102D3000FFFFFFFFFFFFFFFFFFFFFFFFFC02AAAA4D
:102D4000AAAAAAAA0AAAAAAAFFFFFFFFFFFFFFFFDB
:102D5000FFFFFFFFFFFFFFFFFFFC03FFFFFFFFFF82
:102D6000FFFFFFFFFFFFFFFFFC02AAAAAAAAAAAA71
:102D700082AAAAAAFFFFFFFFFFFFFFFFFFFFFFFFDF
:102D8000FFFFFFFFFFFC03FFFFFFFFFFFFFFFFFF52
:102D9000FFFFFFFFFC02AAAAAAAAAAAA82AAAAAABD
:102DA000FFFFFFFFFFFFFFFFFFFFFFFFFFFFFFFF33
:102DB000FFFC03FFFFFFFFFFFFFFFFFFFFFFFFFF22
:102DC000FC02AAAAAAAAAAAA82AAAAAAFFFFFFFF8D
:102DD000FFFFFFFFFFFFFFFFFFFFFFFFFFFC03FF02
:102DE000FFFFFFF00000000FFFFFFFFFFC02AAAA99
:102DF000AAAAAAAA82AAAAAAFFFFFFFFFFFFFFFFB3
:102E0000FFFFFFFFFFFFFFFFFFFC03FFFFFFF000DF
:102E1000000000003FFFFFFFFC02AAAAAAAAAAA086
:102E200002AAAAAAFFFFFFFFFFFFFFFFFFFFFFFFAE
:102E3000FFFFFFFFFFFC03FFFFFF0000000000009B
:102E400003FFFFFFFC02AAAAAA8000000AAAAAAAFE
:102E5000FFFFFFFFFFFFFFFFFFFFFFFFFFFFFFFF82
:102E6000FFFC03FFFFFC000000000000003FFFFF2D
:102E7000FC02AAAAAA800000AAAAAAAAFFFFFFFF32
:102E8000FFFFFFFFFFFFFFFFFFFFFFFFFFFC03FF51
:102E9000FFF0000000000000000FFFFFFC02AAAAE4
:102EA000AAAAAAAAAAAAAAAAFFFFFFFFFFFFFF00D9
:102EB0000000000000000003FFFC03FFFFC0000053
:102EC0000FFFFFF00003FFFFFC02AAAAAAAAAAAA0A
:102ED000AAAAAAAAFFFFFFFFFFFFC0000000000090
:102EE00000000003FFFC03FFFF0003C003FFFFFF20
:102EF000C000FFFFFC02AAAAAAAAAAAAA2AAAAAA7A
:102F0000FFFFFFFFFFFC00000000000000000003C7
:102F1000FFFC03FFFC003FF000FFFFFFFC00FFFF92
:102F2000FC02AAAAAAAAAAA802AAAAAAFFFFFFFFAD
:102F3000FFC000000000000000000003FFFC03FFD2
:102F4000FC00FFFC003FFFFFFF003FFFFC02AAAABE
:102F5000AAAAAA0002AAAAAAFFFFFFFFFF00000078
:102F60000000000000000003FFFC03FFFC03FFFF64
:102F7000003FFFFFFFC03FFFFC02AAAAAAAA8000F1
:102F80002AAAAAAAFFFFFFFFF00000000000C0006D
:102F900000000003FFFC03FFF003FFFF000FFFFF33
:102FA000FFC03FFFFC02AAAAAAA00002AAAAAAAADE
:102FB000FFFFFFFFC0000000000FFC000000000347
:102FC000FFFC03FFF00FFFFFC003FFFFFFF00FFF49
:102FD000FC02AAAAA8000A82AAAAAAAAFFFFFFFFC7
:102FE0000000000000FFFFC000000003FFFC03FF23
:102FF000F00FFFFFF000FFFFFFF00FFFFC02AAAA97
:103000008002AA82AAAAAAAAFFFFFFFC0000000071
:103010000FFFFFFC00000003FFFC03FFF00FFFFFAA
:10302000FC00FFFFFFF00FFFFC02AAAA80AAAA8201
:10303000AAAAAAAAFFFFFFF000000000FFFFFFFFFF
:10304000FC000003FFFC03FFF00FFFFFFC003FFF4D
:10305000FFF00FFFFC02AAAA802AAA82AAAAAAAAA3
:10306000FFFFFFC00000000FFFF000FFFF000003A4
:10307000FFFC03FFF00FFFFFFF000FFFFFF00FFF4C
:10308000FC02AAAA8000AA82AAAAAAAAFFFFFF009D
:10309000000000FFFF00000FFF000003FFFC03FF24
:1030A000FC03FFFFFFC00FFFFFC00FFFFC02AAAA37
:1030B000AA000282AAAAAAAAFFFFFF00000003FF3B
:1030C000FF000000FFC00003FFFC03FFFC03FFFF45
:1030D000FFF003FFFFC03FFFFC02AAAAAAA800025C
:1030E000AAAAAAAAFFFFFC00000003FFFF0000003D
:1030F000FFF00003FFFC03FFFC00FFFFFFF000FFF9
:10310000FF003FFFFC02AAAAAAAAA0000AAAAAAA34
:10311000FFFFFC00000000FFFFC0000000000003F4
:10312000FFFC03FFFF003FFFFFFC003FF0003FFFFD
:10313000FC02AAAAAAAAAA8002AAAAAAFFFFF000D1
:103140000000000FFFFC000000000003FFFC03FF75
:10315000FF0003FFFFFF003FC000FFFFFC02AAAA21
:10316000AAAAAAAA82AAAAAAFFFFF0000000000049
:10317000FFFFC00000000003FFFC03FFFFC0000FC3
:10318000FFFF00000003FFFFFC02AAAAAAAAAAAA46
:10319000AAAAAAAAFFFFC000000000000FFFFC00BF
:1031A00000000003FFFC03FFFFF000000000000030
:1031B0000003FFFFFC02AAAAAAAAAAAAAAAAAAAA6C
:1031C000FFFFC00000000000003FFFF00000000310
:1031D000FFFC03FFFFFC000000000000003FFFFFBA
:1031E000FC02AAAAAAAAAAAAAAAAAAAAFFFFC0007F
:1031F00000000000000FFFF000000003FFFC03FFD1
:10320000FFFFC0000000000000FFFFFFFC02AAAAB1
:10321000AAAAAAAAAAAAAAAAFFFF000003FFF0006E
:10322000000FFFF000000003FFFC03FFFFFFFC00A6
:10323000000000000FFFFFFFFC02AAAAAAAAAAAA88
:10324000AAAAAAAAFFFF000000FFF000000FFFF0EB
:1032500000000003FFFC03FFFFFFFFF00000000F72
:10326000FFFFFFFFFC02AAAAAAAAAAAAAAAAAAAAC0
:10327000FFFF0000003FFFC003FFFF00000000034E
:10328000FFFC03FFFFFFFFFFFFFFFFFFFFFFFFFF4D
:10329000FC02AAAAAAAAAAAAAAAAAAAAFFFF00008E
:1032A000000FFFFC0FFF000000000003FFFC03FF06
:1032B000FFFFFFFFFFFFFFFFFFFFFFFFFC02AAAAC8
:1032C000AAAAAAAAAAAAAAAAFFFF00000003FFFFAF
:1032D000FFFC000000000003FFFC03FFFFFFFFFFF7
:1032E000FFFFFFFFFFFFFFFFFC02AAAAAAAAAAAAEC
:1032F000AAAAAAAAFFFF0000000003FFFFFC00002B
:1033000000000003FFFC03FFFFFFFFFFFFFFFFFFC5
:10331000FFFFFFFFFC02AAAAAAAAAAAAAAAAAAAA0F
:10332000FFFF00000000000FFFFC00000000000392
:10333000FFFC03FFFFFFFFFFFFFFFFFFFFFFFFFF9C
:10334000FC02AAAAAAAAAAAAAAAAAAAAFFFF0000DD
:1033500000000000FFFFC00000000003FFFC03FFAF
:10336000FFFFFFFFFFFFFFFFFFFFFFFFFC02AAAA17
:10337000AAAAAAAAAAAAAAAAFFFF000000000000FF
:103380000FFFFC0000000003FFFC03FFFFFFFFFF37
:10339000FFFFFFFFFF003FFFFC02AAAAAAAAAAAAFA
:1033A000AAAAAAAAFFFF00000000000003FFFFF086
:1033B00000000003FFFC03FFFFFFFFFFFFFFFFFF15
:1033C000FF003FFFFC02AAAAAAAAAAAAAAAAAAAA1E
:1033D000FFFF00000000000003FFFFF000000003FB
:1033E000FFFC03FFFFFFFFFFFFFFFFFFFF003FFFAB
:1033F000FC02AAAAAAAAAAAAAAAAAAAAFFFF00002D
:103400000000000003FFFFF000000003FFFC03FFCB
:10341000FFFFFFFFFFFFFFFFFF003FFFFC02AAAA25
:10342000AAAAAAAAAAAAAAAAFFFF0000000000004E
:10343000FFFFFC0000000003FFFC03FFFFFFFFFF96
:10344000FFFFFFFFFF003FFFFC02AAAAAAAAAAAA49
:10345000AAAAAAAAFFFF00000000003FFFFF000089
:1034600000000003FFFC03FFFFFFFFFFFFFFFFFF64
:10347000FF003FFFFC02AAAAAAAAAAAAAAAAAAAA6D
:10348000FFFF0000000003FFFFF00000000000034A
:10349000FFFC03FFFFFFFFFFFFFFFFFFFF003FFFFA
:1034A000FC02AAAAAAAAAAAAAAAAAAAAFFFF00007C
:1034B000000003FFFF0000000000000FFFFC03FFFF
:1034C000FFFFFFFFFFFFFFFFFF003FFFFC02AAAA75
:1034D000AAAAAAAAAAAAAAAAFFFF0000000003FF9C
:1034E000FF0000000000000FFFFC03FFFC000000D5
:1034F0000000000000003FFFFC02AAAAAAAAAAAA94
:10350000AAAAAAAAFFFF0000000000FFFF00000017
:103510000000000FFFFC03FFFC00000000000000A3
:1035200000003FFFFC02AAAAAAAAAAAAAAAAAAAABB
:10353000FFFF000000000003FFFC00000000003F50
:10354000FFFC03FFFC0000000000000000003FFF44
:10355000FC02AAAAAAAAAAAAAAAAAAAAFFFF0000CB
:10356000000000000FFFF0000000003FFFFC03FF21
:10357000FC0000000000000000003FFFFC02AAAABF
:10358000AAAAAAAAAAAAAAAAFFFF000000000000ED
:103590000FFFFFC0000000FFFFFC03FFFC00000066
:1035A0000000000000003FFFFC02AAAAAAAAAAAAE3
:1035B000AAAAAAAAFFFF0000000000000FFFFFF068
:1035C000000000FFFFFC03FFFC0000000000000003
:1035D00000003FFFFC02AAAAAAAAAAAAAAAAAAAA0B
:1035E000FFFF0000000000003FFFFFF0000003FFAE
:1035F000FFFC03FFFF00FFFFFFFFFFFFFF003FFF98
:10360000FC02AAAAAAAAAAAAAAAAAAAAFFFF00001A
:103610000000000FFFFFFFC000000FFFFFFC03FFD3
:10362000FFC03FFFFFFFFFFFFF003FFFFC02AAAA12
:10363000AAAAAAAAAAAAAAAAFFFF0000000000FF3D
:10364000FFFFF00000000FFFFFFC03FFFFC00FFFB4
:10365000FFFFFFFFFF003FFFFC02AAAAAAAAAAAA37
:10366000AAAAAAAAFFFF0000000003FFFFFC0000B7
:1036700000003FFFFFFC03FFFFF00FFFFFFFFFFF16
:10368000FF003FFFFC02AAAAAAAAAAAAAAAAAAAA5B
:10369000FFFF0000000003FFFF0000000000FFFF2D
:1036A000FFFC03FFFFF003FFFFFFFFFFFF003FFFF3
:1036B000FC02AAAAAAAAAAAAAAAAAAAAFFFF00006A
:1036C000000003FFC00000000003FFFFFFFC03FF3A
:1036D000FFFC00FFFFFFFFFFFF003FFFFC02AAAA65
:1036E000AAAAAAAAAAAAAAAAFFFF0000000003F099
:1036F00000000000000FFFFFFFFC03FFFFFC00FFC6
:10370000FFFFFFFFFF003FFFFC02AAAAAAAAAAAA86
:10371000AAAAAAAAFFFF0000000000000000000003
:10372000003FFFFFFFFC03FFFFFF003FFFFFFFFF26
:10373000FF003FFFFC02AAAAAAAAAAAAAAAAAAAAAA
:10374000FFFF0000000000000000000003FFFFFF7B
:10375000FFFC03FFFFFFC00FFFFFFFFFFF003FFF66
:10376000FC02AAAAAAAAAAAAAAAAAAAAFFFF0000B9
:1037700000000000000000000FFFFFFFFFFC03FF40
:10378000FFFFC03FFFFFFFFFFF003FFFFC02AAAAB1
:10379000AAAAAAAAAAAAAAAAFFFF000000000000DB
:1037A00000000000FFFFFFFFFFFC03FFFFFFF3FF30
:1037B000FFFFFFFFFFFFFFFFFC02AAAAAAAAAAAA17
:1037C000AAAAAAAAFFFF0000000000000000000F44
:1037D000FFFFFFFFFFFC03FFFFFFFFFFFFFFFFFFF8
:1037E000FFFFFFFFFC02AAAAAAAAAAAAAAAAAAAA3B
:1037F000FFFF000000000000000003FFFFFFFFFFCD
:10380000FFFC03FFFFFFFFFFFFFFFFFFFFFFFFFFC7
:10381000FC02AAAAAAAAAAAAAAAAAAAAFFFFFFFF0A
:10382000FFFFFFFFFFFFFFFFFFFFFFFFFFFC03FFA7
:10383000FFFFFFFFFFFFFFFFFFFFFFFFFC02AAAA42
:10384000AAAAAAAAAAAAAAAAFFFFFFFFFFFFFFFF30
:10385000FFFFFFFFFFFFFFFFFFFC03FFFFFFFFFF77
:10386000FFFFFFFFFFFFFFFFFC02AAAAAAAAAAAA66
:10387000AAAAAAAAFFFFFFFFFFFFFFFFFFFFFFFFAC
:10388000FFFFFFFFFFFC03FFFFFFFFFFFFFFFFFF47
:10389000FFFFFFFFFC02AAAAAAAAAAAAAAAAAAAA8A
:1038A000FFFFFFFFFFFFFFFFFFFFFFFFFFFFFFFF28
:1038B000FFFC03FFFFFFFFFFFFFFFFFFFFFFFFFF17
:1038C000FC02AAAAAAAAAAAAAAAAAAAAFFFFFFFF5A
:1038D000FFFFFFFFFFFFFFFFFFFFFFFFFFFC03FFF7
:1038E000FFFFFFFFFFFFFFFFFFFFFFFFFC02AAAA92
:1038F000AAAAAAAAAAAAAAAAFFFFFFFFFFFFFFFF80
:10390000FFFFFFFFFFFFFFFFFFFC03FFFFFFFFFFC6
:10391000FFFFFFFFFFFFFFFFFC02AAAAAAAAAAAAB5
:10392000AAAAAAAAFFFFFFFFFFFFFFFFFFFFFFFFFB
:10393000FFFFFFFFFFFC03FFFFFFFFFFFFFFFFFF96
:10394000FFFFFFFFFC02AAAAAAAAAAAAAAAAAAAAD9
:10395000FFFFFFFFFFFFFFFFFFFFFFFFFFFFFFFF77
:10396000FFFC03FFFFFFFFFFFFFFFFFFFFFFFFFF66
:10397000FC02AAAAAAAAAAAAAAAAAAAAFFFFFFFFA9
:10398000FFFFFFFFFFFFFFFFFFFFFFFFFFFC03FF46
:10399000FFFFFFFFFFFFFFFFFFFFFFFFFC02AAAAE1
:1039A000AAAAAAAAAAAAAAAAFFFFFFFFFFFFFFFFCF
:1039B000FE1FFFFFFFFFFFFFE1FFFFFFFFFFFFFF16
:1039C000FFFFFFFFFFFFFE1FFFFFFFFFFFFFE1FF06
:1039D000FFFFFFFFFFFFFFFFFFFFFFFFFE1FFFFFD8
:1039E000FFFFFFFFE1FFFFFFFFFFFFFFFFFFFFFF05
:1039F000FFFFFE1FFFFFFFFFFFFFE1FFFFFFFFFFD6
:103A0000FFFFFFFFFFFFFFFFFE1FFFFFFFFFFFFFA7
:103A1000E1FFFFFFFFFFFFFFFFFFFFFFFFFFFE1FB5
:103A2000FFFFFFFFFFFFE1FFFFFFFFFFFFFFFFFFC4
:103A3000FFFFFFFFFE1FFFFFFFFFFFFFE1FFFFFF95
:103A4000FFFFFFFFFFFFFFFFFFFFFE1FFFFFFFFF67
:103A5000FFFFE1FFFFFFFFFFFFFFFFFFFFFFFFFF94
:103A6000FE1FFFFFFFFFFFFFE1FFFFFFFFFFFFFF65
:103A7000FFFFFFFFFFFFFE1FFFFFFFFFFFFFE1FF55
:103A8000FFFFFFFFFFFFFFFFFFFFFFFFFE1F8000A5
:103A900000000003E1FFFFFFFFFFFFFFFFFFFFFF4D
:103AA000FFFFFE1F800000000003E1FFFFFFFFFF9C
:103AB000FFFFFFFFFFFFFFFFFE1F8000000000036E
:103AC000E1FFFFFFFFFFFFFFFFFFFFFFFFFFFE1F05
:103AD000800000000003E1FFFFFFFFFFFFFFFFFF8B
:103AE000FFE0FFFFFE1F800000000003E1FFFFFF7B
:103AF000FFFFFFFFFFFFFF801FFFFE1F83FFFFFF92
:103B0000FF83E1FFFFFFFFFFFFFFFFFFFE000FFF4F
:103B1000FE1F83FFFFFFFF83E1FFFFFFFFFFFFFFAC
:103B2000FFFFFC0E07FFFE1F83FFFFFFFF83E1FF88
:103B3000FFFFFFFFFFFFFFFFF83F83FFFE1F83FF35
:103B4000FFFFFF83E1FFFFFFFFFFFFFFFFFFF07FAE
:103B5000E1FFFE1F83FFFFFFFF83E1FFFFFFFFFF8A
:103B6000FFFFFFFFC0FFF1FFFE1F83FFC0000183C7
:103B7000E1FFFFFFFFFFFFFFFFFF01FFF1FFFE1F60
:103B8000830000000183E1FFFFFFFFFFFFFFFFFC59
:103B900001FFF0FFFE1F830000000183E1FFFFFF34
:103BA000FFFFFFFFFFF003FFF0FFFE1F8300000099
:103BB0000183E1FFFFFFFFFFFFFFFFF07FFFF0FF4B
:103BC000FE1F830000000183E1FFFFFFFFFFFFFFF7
:103BD000FFE0FFFFF0FFFE1F8301FFFFFF83E1FF18
:103BE000FFFFFFFFFFFFFFC3FFFFF0FFFE1F83008C
:103BF0003FFFFF83E1FFFFFFFFFFFFFFFFC7FFFF67
:103C0000F0FFFE1F830007FFFF83E1FFFFFFFFFFC1
:103C1000FFFFFF87FFFFF0FFFE1F83E0007FFF83B2
:103C2000E1FFFFFFFFFFFFFFFF8FFFFFF0FFFE1F22
:103C300083FE000FFF83E1FFFFFFFFFFFFFFFF8F0A
:103C4000FFFFF0FFFE1F83FFE003FF83E1FFFFFFA5
:103C5000FFFFFFFFFF8FFFFFF0FFFE1F83FFFE034D
:103C6000FF83E1FFFFFFFFFFFFFFFF8FFFFFF0FF7D
:103C7000FE1F83FFE003FF83E1FFFFFFFFFFFFFF66
:103C8000FF8FFFFFF0FFFE1F83FE0003FF83E1FFB6
:103C9000FFFFFFFFFFFFFF8FFFFFF0FFFE1F83E02F
:103CA000001FFF83E1FFFFFFFFFFFFFFFF87FFFF15
:103CB000F0FFFE1F830001FFFF83E1FFFFFFFFFF17
:103CC000FFFFFF87FFFFF0FFFE1F83001FFFFF8343
:103CD000E1FFFFFFFFFFFFFFFFC3FFFFF0FFFE1F3E
:103CE0008300FFFFFF83E1FFFFFFFFFFFFFFF9C13D
:103CF000FFFFF0FFFE1F830000001F83E1FFFFFFB7
:103D0000FFFFFFFFFCE0FFFFF0FFFE1F830000004E
:103D10000183E1FFFFFFFFFFFFFFFC701FFFF0FFCC
:103D2000FE1F830000000183E1FFFFFFFFFFFFFF95
:103D3000FE381FFFF0FFFE1F830000000183E1FF3C
:103D4000FFFFFFFFFFFFFF3E1FFFF0FFFE1F83FF90
:103D5000C0000183E1FFFFFFFFFFFFFFFFBE1FFF6A
:103D6000F0FFFE1F83FFFFFFFF83E1FFFFFFFFFF69
:103D7000FFFF3FBE1FFFF0FFFE1F83FFFFFFFF831C
:103D8000E1FFFFFFFFFFFFFF0F1E1FFFF0FFFE1F02
:103D900083FFFFFFE183E1FFFFFFFFFFFFFF820ED5
:103DA0001FFFF0FFFE1F83FFFFFF0183E1FFFFFF07
:103DB000FFFFFFFFE01E1FFFF0FFFE1F83FFFFF06E
:103DC0000183E1FFFFFFFFFFFFFFFC3F0FFFF0FF5D
:103DD000FE1F83FFFF800183E1FFFFFFFFFFFFFF67
:103DE000FC3F07FFF0FFFE1F83FFF8000183E1FFA8
:103DF000FFFFFFFFFFFFFC7F81FFF0FFFE1F83FF40
:103E0000C0000183E1FFFFFFFFFFFFFFF87FC00F4E
:103E1000F0FFFE1F83FC00000783E1FFFFFFFFFFB1
:103E2000FFFC007FE01FF0FFFE1F83E000007F83A8
:103E3000E1FFFFFFFFFFFFFC007FFC1FF0FFFE1F05
:103E4000830000007F83E1FFFFFE3FFFFFFFFC7F59
:103E5000FE1FF0FFFE1F830000707F83E1FFFFFC69
:103E60001FFFFFFFFC3FFE1FF0FFFE1F830007F058
:103E70007F83E1FFFFFC1FFFFFFFFC1FFF1FF1FF20
:103E8000FE1F83007FF07F83E1FFFFFE3FFFFFFF08
:103E9000F80FFF0FE1FFFE1F8307FFF07F83E1FFB5
:103EA000FFFFFFFFFFFFF0010F83C1FFFE1F830035
:103EB0007FF07F83E1FFFFFFFFFFFFFFC3800780ED
:103EC00003FFFE1F83000FF07F83E1FFFFFFFFFF73
:103ED000FFFF8FC003C007FFFE1F830000F07F833A
:103EE000E1FFFFFFFFFFFFFF9FC019F01FFFFE1F55
:103EF000838000107F83E1FFFFFFFFFFFFFFFF9E36
:103F00007CFC7FFFFE1F83F000007F83E1FFFFFF4B
:103F1000FFFFFFFFFF9F7C7FFFFFFE1F83FE000070
:103F20003F83E1FFFFFFFFFFFFFFFF3F7E7FFFFFBC
:103F3000FE1F83FFE0000383E1FFFFFFFFFFFFFFA2
:103F4000FF3F7F3FFFFFFE1F83FFFC000183E1FF78
:103F500000001FFFFFFFFE7F3FBFFFFFFE1F83FF2D
:103F6000FFC00183E1FF00001FFFFFFFFFFF3FFFD6
:103F7000FFFFFE1F83FFFFF80183E1FFF8FC7FFFD7
:103F8000FFFFFFFF3FFFFFFFFE1F83FFFFFF0183D8
:103F9000E1FFF9FE3FFFFFFFFFFFFFFFFFFFFE1FF7
:103FA00083FFFFFFF183E1FFF9FF3FFFFFFFFFFF0B
:103FB000FFFFFFFFFE1F83FFFFFFFF83E1FFF9FF0E
:103FC0009FFFFFFFFFFFFFFFFFFFFE1F83FFFFFFBE
:103FD000FF83E1FFF9FF9FFFFFFFFFFFFFFFFFFFF1
:103FE000FE1F83FFFFFFFF83E1FFFCFF9FFFFFFF3B
:103FF000FFFFFFFFFFFFFE1F83FFFFFFFF83E1FFC8
:10400000FC7F1FFFFFFFFFFFFFFFFFFFFE1F800082
:1040100000000003E1FFFE003FFFFFFFFFFFFFFF87
:10402000FFFFFE1F800000000003E1FFFF007FFF95
:10403000FFFFFFFFFFFFFFFFFE1F800000000003E8
:10404000E1FFFFFFFFFFFFFFFFFFFFFFFFFFFE1F7F
:10405000800000000003E1FFFFFFFFFFFFFFFFFF05
:10406000FFFFFFFFFE1F800000000003E1FFFFFFD6
:10407000FFFFFFFFFFFFFFFFFFFFFE1FFFFFFFFF31
:10408000FFFFE1FFFFFFFFFF000000000000000056
:10409000001FFFFFFFFFFFFFE1FFFF07FFFF000023
:1040A000000000000000001FFFFFFFFFFFFFE1FF17
:1040B000FE07BFFF0000000000000000001FFFFF20
:1040C000FFFFFFFFE1FFFC679FFF00000000000013
:1040D0000000001FFFFFFFFFFFFFE1FFF8E79FFF6A
:1040E000FFFFFFFFFFFFFFFFFE1FFFFFFFFFFFFFC1
:1040F000E1FFF9E79FFFFFFFFFFFFFFFFFFFFE1F4D
:10410000FFFFFFFFFFFFE1FFF9E79FFFFFFFFFFF5B
:10411000FFFFFFFFFE1FFFFFFFFFFFFFE1FFF9E7CC
:104120009FFFFFFFFFFFFFFFFFFFFE1FFFFFFFFFE0
:10413000FFFFE1FFF9E71FFFFFFFFFFFFFFFFFFFAB
:10414000FE1FFFFFFFFFFFFFE1FFFCE73FFFFFF860
:1041500003FFFFFFFFFFFE1FFFFFFFFFFFFFE1FF6A
:10416000FC003FFFFFF001FFFFFFFFFFFE1FFFFF0F
:10417000FFFFFFFFE1FFFE007FFFFFC1E03FFFFF0A
:10418000FFFFFE1FFFFFFFFFFFFFE1FFFF81FFFFBC
:10419000FF0FFE1FFFFFFFFFFE1FFFFFFFFFFFFFE1
:1041A000E1FFFFFFFFFFFE3FFF07FFFFFFFFFE1FD7
:1041B000FFFFFFFFFFFFE1FFFFFFFFFFFC3863830F
:1041C000FFFFFFFFFE1FFFFFFFFFFFFFE1FF801F5D
:1041D000FFFFF87031C1FFFFFFFFFE1FFFFFFFFF72
:1041E000FFFFE1FF80001FFFF06030C1FFFFFFFF16
:1041F000FE1FFFFC0003FFFFE1FFFFFC1FFFE0606D
:104200003040FFFFFFFFFE1FFFC000007FFFE1FF08
:10421000FFFE1FFFE060306000000001FE1FFF0096
:1042200000001FFFE1FFFFF07FFFC0703060000063
:104230000001FE1FFE00000007FFE1FFFF83FFFFFC
:10424000C030706000000001FE1FFC00000003FF92
:10425000E1FFFE1FFFFF803FE06000000001FE1F46
:10426000F8003FFC01FFE1FFFE0FFFFF801FC000D1
:1042700000000001FE1FF0181FFF80FFE1FFFFC1DB
:10428000FFFF8003000000000001FE1FE07C0FFF25
:10429000E0FFE1FFFFF83FFF800000001FFFF0019B
:1042A000FE1FE0FE07FFF07FE1FFFFFF1FFF800022
:1042B00000001FFFE001FE1FE1FF07FFF87FE1FFA5
:1042C000E0001FFF800000001FFFC001FE1FC1FFB4
:1042D00003FFF87FE1FF80001FFF8007FC001FFF46
:1042E0008001FE1FC3FF81FFFC3FE1FF83FFFFFF53
:1042F000801FFF001FFF0001FE1FC3FFC0FFFC3F28
:10430000E1FFFFFFFFFF803C67801FFE0081FE1F73
:10431000C3FFE0FFFC3FE1FFFFFFFFFF803021C054
:104320001FFC0181FE1FC3FFE07FFC3FE1FFFFFF99
:10433000FFFFC06030C03FF80381FE1FC3FFF03FA6
:10434000FC3FE1FFFFFFFFFFC06030C07FF00F8147
:10435000FE1FE1FFF83FF83FE1FFFFFFFFFFC060F6
:1043600030607FE01F81FE1FE1FFFC1FF87FE1FF4F
:10437000FFFFFFFFE0603060FFC03F81FE1FE0FFF6
:10438000FC0FF07FE1FFFFFFFFFFE0307060FF8078
:104390007F81FE1FF07FFE07C07FE1FFFFFFFFFF71
:1043A000F038E061FE00FF81FE1FF01FFF0780FF75
:1043B000E1FFFFFFFFFFF81FE061FC01FF81FE1F2F
:1043C000F803FF0001FFE1FFFFFFFFFFFC0F80008C
:1043D000F803FF81FE1FFC00000001FFE1FFFFFF6B
:1043E000FFFFFE0000007007FF81FE1FFE000000BF
:1043F00007FFE1FFFFFFFFFFFF000000200FFF812D
:10440000FE1FFF8000000FFFE1FFFFFFFFFFFF80A7
:104410000060001FFF81FE1FFFE000003FFFE1FF83
:10442000FFFFFFFFFF8001F0003FFF81FE1FFFFC49
:104430000003FFFFE1FFFFFFFFFFFF81FFF800FF29
:10444000FF81FE1FFFFFFFFFFFFFE1FFFFFFFFFFF9
:10445000FF81FFFC01FFFF81FE1FFFFFFFFFFFFF4A
:10446000E1FFFFFFFFFFFF81FFFE01FFFF81FE1F56
:10447000FFFFFFFFFFFFE1FFFFFFFFFFFF81FFFEE9
:1044800001FFFF81FE1FFFFFFFFFFFFFE1FFFFC0F6
:10449000FFFFFF81FFFF00FFFF81FE1FFFFFFFFF08
:1044A000FFFFE1FF9F803FFFFF81FFFF807FFF81D4
:1044B000FE1FFFFFFFFFFFFFE1FF9F9E3FFFFF810A
:1044C000FFFFC03FFF81FE1FFFFC0003FFFFE1FF76
:1044D0009F3F1FFFFF81FFFFE01FFF81FE1FFFC007
:1044E00000007FFFE1FF9F3F9FFFFF81FFFFF00F75
:1044F000FF81FE1FFF0000001FFFE1FF9F3F9FFFA6
:10450000FF81FFFFF80FFF81FE1FFE00000007FF85
:10451000E1FFCF3F9FFFFF81FFFFFC07FF81FE1FF1
:10452000FC00000003FFE1FFCF3F9FFFFF81FFFF83
:10453000FE03FF81FE1FF8003FFC01FFE1FFE39F48
:104540003FFFFF81FFFFFE03FF81FE1FF0181FFFEB
:1045500080FFE1FFF0003FFFFF81FFFFFC03FF81D1
:10456000FE1FE07C0FFFE0FFE1FFF8007FFFFF810F
:10457000FFFFF807FF81FE1FE0FE07FFF07FE1FF6E
:10458000FF03FFFFFF81FFFFF00FFF81FE1FE1FF31
:1045900007FFF87FE1FFFFFFFFFFFF81FFFFE01F45
:1045A000FF81FE1FC1FF03FFF87FE1FFFFFFFFFF59
:1045B000FF81FFFFC03FFF81FE1FC3FF81FFFC3F64
:1045C000E1FFFFFFFFFFFF81FFFFC07FFF81FE1FB5
:1045D000C3FFC0FFFC3FE1FFFFFF9FFFFF81FFFF25
:1045E00080FFFF81FE1FC3FFE0FFFC3FE1FFFFFFF5
:1045F0009FFFFF81FFFF01FFFF81FE1FC3FFE07FE1
:10460000FC3FE1FFFFFF9FFFFF81FFFE01FFFF81F6
:10461000FE1FC3FFF03FFC3FE1FFFFFF9FFFFF8155
:10462000FFFC01FFFF81FE1FE1FFF83FF83FE1FFC4
:1046300080001FFFFF81FFF800FFFF81FE1FE1FFE9
:10464000FC1FF87FE1FF80001FFFFF81FFF0007F6C
:10465000FF81FE1FE0FFFC0FF07FE1FF80001FFFE6
:10466000FF81FFE0003FFF81FE1FF07FFE07C07F5C
:10467000E1FFDFFF9FFFFF81FFE0001FFF81FE1FC3
:10468000F01FFF0780FFE1FFCFFF9FFFFF81FFC00B
:10469000700FFF81FE1FF803FF0001FFE1FFE7FF3E
:1046A0009FFFFF81FF80F807FF81FE1FFC000000D5
:1046B00001FFE1FFE7FF9FFFFF81FF01FC01FF8199
:1046C000FE1FFE00000007FFE1FFF7FF9FFFFF81D5
:1046D000FE01FE00FF81FE1FFF8000000FFFE1FFD3
:1046E000FFFFFFFFFF81FC03FF007F81FE1FFFE054
:1046F00000003FFFE1FFFFFFFFFFFF81F807FF80A2
:104700003F81FE1FFFFC0003FFFFE1FFFFFFFFFFF4
:10471000FF81F00FFFC01F81FE1FFFFFFFFFFFFFA4
:10472000E1FFFFFFFFFFFF81E01FFFE00F81FE1FA2
:10473000FFFFFFFFFFFFE1FFFFFFFFFFFF81E03F04
:10474000FFF00781FE1FFFFFFFFFFFFFE1FFFFFFFD
:10475000FFFFFF81C07FFFFC0381FE1FFFFFFFFF04
:10476000FFFFE1FFFFFFFFFFFF8180FFFFFE0181F1
:10477000FE1FFFFFFFFFFFFFE1FFFFFFFFFFFF81C6
:1047800000FFFFFF0081FE1FFFFFFFFFFFFFE1FFB4
:10479000FFFFFFFFFF8001FFFFFF8001FE1FFFFF04
:1047A000FFFFFFFFE1FFFFFFFFFFFF8003FFFFFFB2
:1047B000C001FE1FFFFFFFFFFFFFE1FFFFFFFFFF45
:1047C000FF8007FFFFFFE001FE1FFFFFFFFFFFFF6E
:1047D000E1FFFFFFFFFFFF800FFFFFFFF001FE1F64
:1047E000FFFFFFFFFFFFE1FFFFFFFFFFFF800FFF66
:1047F000FFFFF001FE1FFFFFFFFFFFFFE1FFFFFFD5
:10480000FFFFFF80000000000001FE1FFFFFFFFF11
:10481000FFFFE1FFFFFFFFFFFF800000000000013E
:10482000FE1FFFFFFFFFFFFFE1FFFFFFFFFFFF8016
:10483000000000000001FE1FFFFFFFFFFFFFE1FF80
:10484000FFFFFFFFFF80000000000001FE1FFFFFD1
:10485000FFFFFFFFE1FFFFFFFFFFFF800000000001
:104860000001FE1FFFFC7FFFF1FFE1FFF9FFE7FF03
:10487000FFFFFFFFFFFFFFFFFE1FFFF01FFFC07FD7
:10488000E1FFF9FFC3FFFFFFFFFFFFFFFFFFFE1F79
:10489000FFF01FFFC07FE1FFF80F81FFFFFFFFFF69
:1048A000FFFFFFFFFE1FFFE00FFF803FE1FFF80764
:1048B00099FFFFFFFFFFFFFFFFFFFE1FFFE00FFF5E
:1048C000803FE1FFF8E79CFFFFFFFFFFFFFFFFFFD7
:1048D000FE1FFFE00FFF803FE1FFF9F39CFFFFFFAA
:1048E000FFFFFFFFFFFFFE1FFFF01FFFC07FE1FF85
:1048F000F9F39CFFFFFFFFFFFFFFFFFFFE1FFFF02D
:104900001FFFC07FE1FFF9F39CFFFFFFFFFFFFFFE9
:10491000FFFFFE1FFFFC7FFFF1FFE1FFF9F39CFFAC
:10492000FFFFFFFFFFFFFFFFFE1FFFFFFFFFFFFF78
:10493000E1FFFCE79CFFFFFFFFFFFFFFFFFFFE1F04
:10494000FFFFFFFFFFFFE1FFFC0009FFFFFFFFFF8D
:10495000FFFFFFFFFE1FFFFFFFFFFFFFE1FFFE085E
:1049600001FFFFFFFFFFFFFFFFFFFE1FFFFFFFFF36
:10497000FFFFE1FFFFFC61FFFFFFFFFFFFFFFFFF06
:10498000FE1FFFFFFFFFFFFFE1FFFFFFFFFFFFFF36
:10499000FFFFFFFFFFFFFE1FFFFFFFFFFFFFE1FF26
:1049A000FFFFFFFF0000000000000000001FFFFFEE
:1049B000FFFFFFFFE1FFFFFFFFFF0000000000001F
:1049C0000000001FFFFFFFFFFFFFE1FFFFFFFFFFF2
:1049D0000000000000000000001FFFFFFFFFFFFFBE
:1049E000E1FFF8001FFF0000000000000000001FB2
:1049F000FFFFFFFFFFFFE1FFF8001FFFFFFFFFFFCB
:104A0000FFFFFFFFFE1FFFFFFFFFFFFFE1FFFFFEB6
:104A10007FFFFFFFFFFFFFFFFFFFFE1FFFFFFFFF07
:104A2000FFFFE1FFFFFF3FFFFFFFFFFFFFFFFFFF74
:104A3000FE1FFFFFFFFFFFFFE1FFFFFF9FFFFFFFE5
:104A4000FFFFFFFFFFFFFE1FFFFFFFFFFFFFE1FF75
:104A5000FFFF9FFFFFFFFFFFFFFFFFFFFE1FFFFFA7
:104A6000FFFFFFFFE1FFFFFF9FFFFFFFFFFFFFFFD4
:104A7000FFFFFE1FFFFC0003FFFFE1FFFFFF9FFFA3
:104A8000FFFFFFFFFFFFFFFFFE1FFFC000007FFFD4
:104A9000E1FFFFFC1FFFFFFFFFFFFFFFFFFFFE1F08
:104AA000FF0000001FFFE1FFF8003FFFFFFFFFFFD7
:104AB000FFFFFFFFFE1FFE00000007FFE1FFF80001
:104AC000FFFFFFFFFFFFFFFFFFFFFE1FFC000000D7
:104AD00003FFE1FFFFFFFFFFFFFFFFF0000000010A
:104AE000FE1FF8003FFC01FFE1FFFFFFFFFFFFFF9C
:104AF000FF8000000001FE1FF0181FFF80FFE1FF94
:104B0000FFFFDFFFFFFFFE0000000001FE1FE07C53
:104B10000FFFE0FFE1FFFFFE1FFFFFFFF8000000B7
:104B20000001FE1FE0FE07FFF07FE1FFFFF01FFF27
:104B3000FFFFF00000000001FE1FE1FF07FFF87F0C
:104B4000E1FFFF807FFFFFFFC00000800001FE1F2C
:104B5000C1FF03FFF87FE1FFFC01FFFFFFFF8000C3
:104B600003E00001FE1FC3FF81FFFC3FE1FFE039CE
:104B7000FFFFFFFF00000FF80001FE1FC3FFC0FF93
:104B8000FC3FE1FF81F9FFFFFFFE00003FFE000157
:104B9000FE1FC3FFE0FFFC3FE1FF8FF9FFFFFFFCBB
:104BA0000000FFFFE001FE1FC3FFE07FFC3FE1FFCD
:104BB00087F9FFFFFFF80003FC0FF001FE1FC3FFA2
:104BC000F03FFC3FE1FF80F9FFFFFFF0000FF00333
:104BD000F001FE1FE1FFF83FF83FE1FFF019FFFF92
:104BE000FFF0001FF000F801FE1FE1FFFC1FF87F3F
:104BF000E1FFFE01FFFFFFE0001FF000FC01FE1FD0
:104C0000E0FFFC0FF07FE1FFFFC03FFFFFE0000F80
:104C1000F8000001FE1FF07FFE07C07FE1FFFFF8F4
:104C20001FFFFFC00003FE000001FE1FF01FFF0773
:104C300080FFE1FFFFFF9FFFFFC00000FF8000013A
:104C4000FE1FF803FF0001FFE1FFFFFFFFFFFF80F2
:104C500000003FE00001FE1FFC00000001FFE1FF3B
:104C6000FFFFFFFFFF80000007FC0001FE1FFE00AA
:104C7000000007FFE1FFFFFFFFFFFF80000003FCD4
:104C80000001FE1FFF8000000FFFE1FFFFFFFFFF9D
:104C9000FF001FC003FC0001FE1FFFE000003FFFFC
:104CA000E1FFFFFFFFFFFF000FC003FC0001FE1F3D
:104CB000FFFC0003FFFFE1FFFFFFFFFFFF0007F81E
:104CC0001FF00001FE1FFFFFFFFFFFFFE1FFFFFFDF
:104CD000FFFFFF0003FE3F000001FE1FFFFFFFFF7D
:104CE000FFFFE1FFFFFFFFFFFF0001FFFE000001EC
:104CF000FE1FFFFFFFFFFFFFE1FFFFFFFFFFFF00C2
:104D0000001FFE000001FE1FFFFFFFFFFFFFE1FF8E
:104D1000FFFFFFFFFF000003FE000001FE1FFFFF7B
:104D2000FFFFFFFFE1FFFFFFFFFFFF000000FF802D
:104D30000001FE1FFFFFFFFFFFFFE1FFFFFFFFFF7F
:104D4000FF0000003FE00001FE1FFFFFFFFFF07FBC
:104D5000E1FFFFFFFFFFFF0000001FFC0001FE1F3F
:104D6000FFFFFFFFF07FE1FFFFFFFFFFFF000000FD
:104D70001FFC0001FE1FFFFFFFFFF07FE1FFFFFFB1
:104D8000FFFFFF0000001FFC0001FE1FFFFFFFFFF1
:104D9000F07FE1FFFFFFFFFFFF000000FFE00001E9
:104DA000FE1FFFFFFFFFF07FE1FFFFFFFFFFFF00A0
:104DB0000007FF000001FE1FFFFFFFFFF07FE1FF84
:104DC000FFFFFFFFFF00001FFC000001FE1FFFFFB1
:104DD000FFFFF07FE1FFFFFFFFFFFF00001FF0007C
:104DE0000003FE1FFFFFFFFFF07FE1FFFFFFFFFF5C
:104DF000FF00001FF0000003FE1FE0000000007F26
:104E0000E1FFFFFFFFFFFF00000FF0000003FE1FA8
:104E1000E0000000007FE1FFFFFFFFFFFF00000157
:104E2000FE000007FE1FE0000000007FE1FFFFFF23
:104E3000FFFFFF0000003FC00007FE1FE000000072
:104E4000007FE1FFFFFFFFFFFF0000003FF8000FC2
:104E5000FE1FE0000000007FE1FFFFFFFFFFFF00FB
:104E600000003FFC000FFE1FE0000000007FE1FF9C
:104E7000FFFFFFFFFF0000007FFC001FFE1FF0FF91
:104E8000FFFFF07FE1FFFFFFFFFFFF000003FFF8E0
:104E9000003FFE1FF87FFFFFF07FE1FFFFFFFFFFF6
:104EA000FF00000FFFC0003FFE1FF83FFFFFF07F35
:104EB000E1FFFFFFFFFFFF00001FFE00007FFE1F5E
:104EC000FC3FFFFFF07FE1FFFFFFFFFFFF00001F40
:104ED000F00000FFFE1FFC1FFFFFF07FE1FFFFFF60
:104EE000FFFFFF00001F800001FFFE1FFE0FFFFFFE
:104EF000F07FE1FFFFFFFFFFFF00001C000003FF4A
:104F0000FE1FFE0FFFFFF07FE1FFFFFFFFFFFF002F
:104F10000000000007FFFE1FFF07FFFFF07FE1FF1B
:104F2000FFFFFFFFFF00000000001FFFFE1FFF83C9
:104F3000FFFFF07FE1FFFFFFFFFFFF000000000029
:104F40003FFFFE1FFF87FFFFF07FE1FFFFFFFFFF37
:104F5000FF0000000000FFFFFE1FFFDFFFFFFFFF5D
:104F6000E1FFFFFFFFFFFF0000000003FFFFFE1F48
:104F7000FFFFFFFFFFFFE1FFFFFFFFFFFF0000005C
:104F8000001FFFFFFE1FFFFFFFFFFFFFE1FFFFFF0F
:104F9000FFFFFFFFFFFFFFFFFFFFFE1FFFFFFFFF02
:104FA000FFFFE1FFFFFFFFFFFFFFFFFFFFFFFFFF2F
:104FB000FE1FFFFFFFFFFFFFE1FFFFFFFFFFFFFF00
:104FC000FFFFFFFFFFFFFE1FFFFFFFFFFFFFE1FFF0
:104FD000FFFFFFFFFFFFFFFFFFFFFFFFFE1FFFFFC2
:104FE000FFFFFFFFE1FFFFFFFFFFFFFFFFFFFFFFEF
:104FF000FFFFFE1FFFFFFFFFFFFFE1FFFFFFFFFFC0
:10500000FFFFFFFFFFFFFFFFFE1FFFFFFFFFFFFF91
:10501000E1FFFFFFFFFFFFFFFFFFFFFFFFFFFE1F9F
:10502000FFFFFFFFFFFFE1FFFFFFFFFFFFFFFFFFAE
:10503000FFFFFFFFFE1FFFFFFFFFFFFFE1FFFFFF7F
:10504000FFFFFFFFFFFFFFFFFFFFFE1FFFFFFFFF51
:10505000FFFFE1FFFFFFFFFF00000000240027002B
:105060002A0000000000250028002B00000000009E
:10507000230026002900040404040404040402029A
:1050800002020202030303030303010204081020C7
:1050900040800102040810200102040810200000D2
:1050A00000080002010000030407000000000000E7
:1050B0000000553311241FBECFEFD8E0DEBFCDBFB7
:1050C00013E0A0E0B1E0E4E6F7E602C005900D923F
:1050D000AA31B107D9F723E0AAE1B3E001C01D92DC
:1050E000A53CB207E1F718E2CAE5D8E204C021976F
:1050F000FE010E94AA33C935D107C9F70E943A328E
:105100000C94B0330C940000AF92BF92CF92DF9218
:10511000EF92FF920F931F93CF93DF936C017B016C
:105120008B01040F151FEB015E01AE18BF08C017FD
:10513000D10759F06991D601ED91FC910190F08170
:10514000E02DC6010995892B79F7C501DF91CF9133
:105150001F910F91FF90EF90DF90CF90BF90AF9095
:105160000895FC01538D448D252F30E0842F90E06D
:10517000821B930B541710F0CF9608950197089552
:10518000FC01918D828D981761F0A28DAE0FBF2F1B
:10519000B11D5D968C91928D9F5F9F73928F90E071
:1051A00008958FEF9FEF0895FC01918D828D9817E0
:1051B00031F0828DE80FF11D858D90E008958FEF1D
:1051C0009FEF0895FC01918D228D892F90E0805CE6
:1051D0009F4F821B91098F739927089588E293E06E
:1051E0000E94E22821E0892B09F420E0822F089513
:1051F00080E090E0892B29F00E94EE2881110C9428
:1052000000000895FC01A48DA80FB92FB11DA35A69
:10521000BF4F2C91848D90E001968F739927848FD6
:10522000A689B7892C93A089B1898C9183708064F9
:105230008C93938D848D981306C00288F389E02D9A
:1052400080818F7D80830895EF92FF920F931F934B
:10525000CF93DF93EC0181E0888F9B8D8C8D981329
:105260001AC0E889F989808185FF15C09FB7F89435
:10527000EE89FF896083E889F98980818370806481
:1052800080839FBF81E090E0DF91CF911F910F91CC
:10529000FF90EF900895F62E0B8D10E00F5F1F4FDB
:1052A0000F731127E02E8C8D8E110CC00FB607FCEA
:1052B000FACFE889F989808185FFF5CFCE010E9478
:1052C0000229F1CFEB8DEC0FFD2FF11DE35AFF4FBB
:1052D000F0829FB7F8940B8FEA89FB898081806206
:1052E000CFCFCF93DF93EC01888D8823B9F0AA89C3
:1052F000BB89E889F9898C9185FD03C0808186FD91
:105300000DC00FB607FCF7CF8C9185FFF2CF8081DF
:1053100085FFEDCFCE010E940229E9CFDF91CF9129
:105320000895833081F028F4813099F08230A9F01B
:1053300008958730A9F08830C9F08430B1F48091A5
:1053400080008F7D03C0809180008F7780938000E4
:10535000089584B58F7784BD089584B58F7DFBCF84
:105360008091B0008F778093B00008958091B00055
:105370008F7DF9CFCF93DF93282F30E0F901E256EC
:10538000FF4A8491F901E657FF4AD491F901EA589E
:10539000FF4AC491CC23A1F081110E949129EC2FE6
:1053A000F0E0EE0FFF1FE459FF4AA591B491EC9194
:1053B000ED2381E090E009F480E0DF91CF91089542
:1053C00080E090E0FACF1F93CF93DF93282F30E057
:1053D000F901E256FF4A8491F901E657FF4AD49158
:1053E000F901EA58FF4AC491CC23A9F0162F811184
:1053F0000E949129EC2FF0E0EE0FFF1FEE59FF4ABB
:10540000A591B4918FB7F894EC91111108C0D09583
:10541000DE23DC938FBFDF91CF911F910895DE2BA8
:10542000F8CFCF93DF9390E0FC01E657FF4A249139
:105430008A589F4AFC0184918823D1F090E0880F1C
:10544000991FFC01E85AFF4AA591B491FC01EE595D
:10545000FF4AC591D49161110EC09FB7F8948C9109
:10546000E22FE0958E238C932881E223E8839FBF6F
:10547000DF91CF9108958FB7F894EC91E22BEC93E4
:105480008FBFF6CF3FB7F894809124039091250306
:10549000A0912603B091270326B5A89B05C02F3FF6
:1054A00019F00196A11DB11D3FBFBA2FA92F982F4A
:1054B0008827BC01CD01620F711D811D911D42E045
:1054C000660F771F881F991F4A95D1F708958F920D
:1054D0009F92AF92BF92CF92DF92EF92FF926B01B9
:1054E0007C010E94422A4B015C01C114D104E104F9
:1054F000F104B9F00E94422A681979098A099B09C6
:10550000683E73408105910580F321E0C21AD108FD
:10551000E108F10888EE880E83E0981EA11CB11CFA
:10552000E4CFFF90EF90DF90CF90BF90AF909F902F
:105530008F900895CF93DF93DC01E90112968D914E
:105540009C911397681779079CF557FD31C0149605
:105550002D913C9115974217530754F5849FF00104
:10556000859FF00D949FF00D1124AF01460F571F3A
:1055700057FF02C0495F5F4F83E0559547958A9575
:10558000E1F7ED91FC91E40FF51F3081CB0168E06C
:1055900070E00E94823340E850E0BA0102C0759585
:1055A00067958A95E2F7CB01CD2B29F0832B808379
:1055B000DF91CF91089580958323F9CFCF93C82FA2
:1055C00060E08AE00E94E329CEBD00000DB407FE32
:1055D000FDCF8EB561E08AE0CF910C94E329BC0148
:1055E00090E080E00C94672ACF93DF93EC0161E0B8
:1055F0008C810E94E32988EC90E00E94EF2A60E011
:105600008C810E94E3298AE090E00E94EF2A61E009
:105610008C810E94E32988EC90E0DF91CF910C947B
:10562000EF2ACF93C62F61E0FC0186810E94E32917
:105630008C2FCF910C94DE2ACF93C62F60E0FC0113
:1056400086810E94E3298C2FCF910C94DE2AFC01E5
:1056500001900020E9F73197AF01481B590BBC01BD
:1056600088E293E00C948428CF93DF93EC018CE6DE
:1056700092E00E94272B8A850E94BA29892B29F45F
:1056800084E690E00E94EF2AF6CF8BE792E0DF916C
:10569000CF910C94272BEF92FF920F931F93CF93F0
:1056A000DF93EC0161E08AE00E94112A61E088E06A
:1056B0000E94112A61E089E00E94112A60E087E0DF
:1056C0000E94112A1FB7F89480911E03811127C0F0
:1056D000E0E8F0E58491E4E9F0E59491E82FF0E06A
:1056E000EE0FFF1FE85AFF4AA591B491EC91E92310
:1056F00021F461E08AE00E94E32961E08AE00E94EF
:10570000112A8CB580618CBD8CB580648CBD61E044
:105710008DE00E94112A61E08BE00E94112A8091A5
:105720001E038F5F80931E031FBF81E58CBD81E048
:105730008DBDCE010E94F42A61E0CE010E941C2B97
:1057400063E0CE010E94112B60E0CE010E94112B7C
:105750006BE2CE010E94112B6BE2CE010E94112B55
:1057600069E0CE010E94112B66E0CE010E941C2B45
:1057700067E0CE010E94112B67E0CE010E94112B41
:1057800067E1CE010E94112B68EFCE010E941C2B15
:1057900060E6CE010E94112B65EACE010E94112B1A
:1057A00068EFCE010E941C2B69E8CE010E94112BEC
:1057B00065EACE010E94112B68EFCE010E941C2BDE
:1057C00060E9CE010E94112B60E0CE010E94112BF6
:1057D00068EFCE010E941C2B63E9CE010E94112BC1
:1057E0006AE2CE010E94112B68EFCE010E941C2BB1
:1057F00060EACE010E94112B65EACE010E94112BB6
:1058000068EFCE010E941C2B61EACE010E94112B91
:1058100060E0CE010E94112B68EFCE010E941C2B8C
:1058200063E7CE010E94112B61E4CE010E94112B8F
:1058300066E1CE010E941C2B60E0CE010E94112B7C
:1058400064E0CE010E941C2BCE010E94342B60E04C
:10585000CE010E941C2B6FEACE010E94112B60E347
:10586000CE010E941C2B6AE3CE010E94112B62E83C
:10587000CE010E941C2B62E1CE010E94112B82E01E
:1058800090E00E94EF2A60E2CE010E941C2B0EE203
:1058900012E0F80161918F01CE010E94112BF2E01C
:1058A0000A351F07B1F761E2CE010E941C2B04E00C
:1058B00012E0F80161918F01CE010E94112BF2E0FC
:1058C0000E321F07B1F762E2CE010E941C2B04E0EA
:1058D00012E08EE2E82E82E0F82EF80161918F014D
:1058E000CE010E94112BE016F106B9F763E2CE015A
:1058F0000E941C2B0AED11E0F80161918F01CE018D
:105900000E94112BF2E004301F07B1F764E2CE01D0
:105910000E941C2B0AED11E0F80161918F01CE016C
:105920000E94112BF2E004301F07B1F790E080E0F5
:10593000DF91CF911F910F91FF90EF9008954F92BB
:105940005F926F927F928F929F92AF92BF92CF920F
:10595000DF92EF92FF920F931F93CF93DF93CDB718
:10596000DEB7C451D4400FB6F894DEBF0FBECDBF32
:1059700088E090E0CB5FDB4F99838883C550D440AB
:1059800089E090E0C95FDB4F99838883C750D4409A
:105990008AE090E0C75FDB4F99838883C950D44089
:1059A00087E090E0C55FDB4F99838883CB50D4407C
:1059B00000EB10E0CF5FDB4F19830883C150D44068
:1059C00088E091E0CD5FDB4F99838883C350D4405A
:1059D00084E00E94BA297C0190931D0380931C03EC
:1059E00085E00E94BA2990931B0380931A03EA94DE
:1059F000EF2809F0CBC1CE018F5F9B4F0E944B2B4C
:105A0000CD5EDB4F19821882C351D440CE0101967E
:105A1000C35FDB4F99838883CD50D440C15FDB4F98
:105A200019830883CF50D44088E190E0CF5EDB4FEC
:105A300099838883C151D44010E000E0C15FDB4FFF
:105A400088819981CF50D440081719070CF499C068
:105A5000A2E94A2EA2E05A2EB12CA12CB0E86B2E5E
:105A6000712CF20181912F01882309F4EEC040913D
:105A7000020150910301BA016770772721E030E0FD
:105A8000672B11F430E020E0F3E056954795FA9546
:105A9000E1F7240F351F6091040170910501269FE5
:105AA000A001279F500D369F500D1124082E000C89
:105AB000990B8097489F9001499F300D589F300D5A
:105AC0001124E0900001F0900101E20EF31E10E0BD
:105AD00000E080910401909105010817190708F072
:105AE000ADC0D12CC12C8091020190910301C81648
:105AF000D90608F099C0F70124914601F7E08F22FA
:105B00009924C301082C02C0959587950A94E2F761
:105B100030E082239323892B49F1C15FDB4F6881F9
:105B20007981CF50D440CF5EDB4F48815981C1513C
:105B3000D440C5018C0D9D1DCD5EDB4F2881398180
:105B4000C351D44021153105B9F597FD0FC0861713
:105B5000970764F4041715074CF430E020E0A8011F
:105B6000BC01CE01835F9B4F0E949A2A87E0881672
:105B7000910419F4EFEFEE1AFE0AFFEFCF1ADF0AD5
:105B8000B2CFF12CE12CCF5EDB4F88819981C151DE
:105B9000D440E816F9066CF421E030E0A701B80122
:105BA000CE01835F9B4F0E949A2AEFEFEE1AFE0A06
:105BB000EACF0F5F1F4F42CF2130310571F497FDBF
:105BC000D5CF8417950794F6061717077CF6601B48
:105BD000710B30E020E0AC01C4CF2230310581F4FC
:105BE00097FDC4CF861797070CF6041715070CF01E
:105BF000BDCF401B510B681B790B30E020E0B1CFCB
:105C00002330310509F0B2CF97FDB0CF8417950747
:105C10000CF0ACCF061717070CF0A8CF481B590B98
:105C200030E020E0B8019DCF87709927892B19F0CB
:105C30008FEFE81AF80A0F5F1F4F4BCF80910201D8
:105C400090910301A80EB91E0CCFC35FDB4FE88013
:105C5000F980CD50D440E114F10409F46EC0CF5E58
:105C6000DB4F08811981C151D440C15FDB4FC8802F
:105C7000CF50D440C05FDB4FD880C051D44065E1E5
:105C8000CE018F5F9B4F0E941C2B60E0CE018F5F87
:105C90009B4F0E94112B60E1CE018F5F9B4F0E94B2
:105CA000112B60E0CE018F5F9B4F0E94112B60E2B1
:105CB000CE018F5F9B4F0E94112B6D2DCE018F5F08
:105CC0009B4F0E94112B6C2D687FCE018F5F9B4FE5
:105CD0000E94112B612FCE018F5F9B4F0E94112BD1
:105CE000602FCE018F5F9B4F0E94112B82E090E0CE
:105CF0000E94EF2AC60197FD0796E3E095958795E8
:105D0000EA95E1F7809F6001819FD00C909FD00CB5
:105D100011248701C8018E199F098C159D054CF42B
:105D2000F80161918F01CE018F5F9B4F0E94112B73
:105D3000F1CF82E090E00E94EF2A8FE992E00E948A
:105D4000272B62E1CE018F5F9B4F0E941C2B88ECBA
:105D500090E00E94EF2ACE018F5F9B4F0E94342B70
:105D600081EB92E00E94272B67E0CE018F5F9B4F73
:105D70000E941C2B65EACE018F5F9B4F0E94112B66
:105D80006DE770E080E090E00E94672A80911A033E
:105D900090911B03019709F0B3C28AEB92E00E9435
:105DA000272BCE018F5F9B4F0E944B2B8CEC92E0F8
:105DB0000E94272B60E1CE018F5F9B4F0E941C2B1E
:105DC00082E090E00E94EF2A00EB16E16FEFCE0137
:105DD0008F5F9B4F0E94112B01501109B9F782E090
:105DE00090E00E94EF2A63E1CE018F5F9B4F0E94FB
:105DF0001C2B82E090E00E94EF2A08EA19E378E584
:105E0000E72E70E5F72EF8016491CE018F5F9B4F6E
:105E10000E94112B0F5F1F4FE016F106A1F782E0E1
:105E200090E00E94EF2A62E1CE018F5F9B4F0E94BB
:105E30001C2B88EC90E00E94EF2ACE018F5F9B4FD5
:105E40000E94342B80EE92E00E94272BCE018F5FC0
:105E50009B4F0E94F42A61E0CE018F5F9B4F0E940E
:105E60001C2B63E0CE018F5F9B4F0E94112B60E0E3
:105E7000CE018F5F9B4F0E94112B6BE2CE018F5F93
:105E80009B4F0E94112B6BE2CE018F5F9B4F0E94B4
:105E9000112B66E0CE018F5F9B4F0E941C2B67E0A9
:105EA000CE018F5F9B4F0E94112B67E0CE018F5F69
:105EB0009B4F0E94112B67E1CE018F5F9B4F0E9489
:105EC000112B68EFCE018F5F9B4F0E941C2B60E669
:105ED000CE018F5F9B4F0E94112B65EACE018F5F31
:105EE0009B4F0E94112B68EFCE018F5F9B4F0E944A
:105EF0001C2B69E8CE018F5F9B4F0E94112B65EA36
:105F0000CE018F5F9B4F0E94112B68EFCE018F5FF8
:105F10009B4F0E941C2B60E9CE018F5F9B4F0E941C
:105F2000112B60E0CE018F5F9B4F0E94112B68EF19
:105F3000CE018F5F9B4F0E941C2B63E9CE018F5FC8
:105F40009B4F0E94112B6AE2CE018F5F9B4F0E94F4
:105F5000112B68EFCE018F5F9B4F0E941C2B60EAD4
:105F6000CE018F5F9B4F0E94112B65EACE018F5FA0
:105F70009B4F0E94112B68EFCE018F5F9B4F0E94B9
:105F80001C2B61EACE018F5F9B4F0E94112B60E0BA
:105F9000CE018F5F9B4F0E94112B68EFCE018F5F68
:105FA0009B4F0E941C2B63E7CE018F5F9B4F0E948B
:105FB000112B61E4CE018F5F9B4F0E94112B66E194
:105FC000CE018F5F9B4F0E941C2B60E0CE018F5F44
:105FD0009B4F0E94112B64E0CE018F5F9B4F0E946C
:105FE0001C2BCE018F5F9B4F0E94342B60E0CE01B3
:105FF0008F5F9B4F0E941C2B6FEBCE018F5F9B4FDF
:106000000E94112B60E3CE018F5F9B4F0E941C2BDF
:1060100060E9CE018F5F9B4F0E94112B61E6CE019C
:106020008F5F9B4F0E941C2B60E0CE018F5F9B4FC8
:106030000E94112B60EBCE018F5F9B4F0E94112BB2
:1060400061E0CE018F5F9B4F0E94112B68E0CE0173
:106050008F5F9B4F0E94112B62E8CE018F5F9B4F99
:106060000E941C2B62E1CE018F5F9B4F0E94112B7F
:1060700060E5CE018F5F9B4F0E941C2B67E9CE012C
:106080008F5F9B4F0E94112B60E1CE018F5F9B4F72
:106090000E941C2B10E000E060E090E080E0A8018E
:1060A000485B534FFA01E80FF91FE4912E2F207C33
:1060B000203C11F0203809F46160660F2E2F220F6A
:1060C000220F207C203C11F0203809F46160660F1B
:1060D0002E2F2295207C203C29F4616005C081E0B0
:1060E00090E0E0CF2038C9F3660FE295EE0FEE0F97
:1060F000E07CE03C11F4616002C0E038E1F3813003
:10610000910509F0660F019751F7CE018F5F9B4F04
:106110000E94112B0E5F1F4F0036FDE21F0709F092
:10612000BBCF63E1CE018F5F9B4F0E941C2B10E021
:1061300000E060E090E080E0D801A85BB34FFD0193
:10614000E80FF91FE49130E020E04E2F407C403C06
:1061500041F4616008C081E090E0F1CF21E030E0DF
:10616000F4CFE6FDF6CF660F4E2F440F440F542FA9
:10617000507C503C11F4616002C046FDFCCF813080
:10618000910519F42130310509F0660FE295E07FA1
:106190002130310519F70197F1F6CE018F5F9B4F42
:1061A0000E94112B0E5F1F4F00368DE2180709F079
:1061B000C0CF60E2CE018F5F9B4F0E941C2B0EEA86
:1061C00011E0F80161918F01CE018F5F9B4F0E941A
:1061D000112BF1E00A3D1F07A1F761E2CE018F5FAD
:1061E0009B4F0E941C2B54E8E52E51E0F52E6EEAE1
:1061F000C62E61E0D62E8701F80161918F01CE0194
:106200008F5F9B4F0E94112BC016D106A9F762E247
:10621000CE018F5F9B4F0E941C2B3AE5C32E31E0CD
:10622000D32E44E8A42E41E0B42EF60161916F0113
:10623000CE018F5F9B4F0E94112BAC14BD04A9F7B8
:1062400063E2CE018F5F9B4F0E941C2B90E3C92E0F
:1062500091E0D92E2AE5A22E21E0B22EF60161911D
:106260006F01CE018F5F9B4F0E94112BAC14BD04B8
:10627000A9F764E2CE018F5F9B4F0E941C2B86E042
:10628000C82E81E0D82EF60161916F01CE018F5F9B
:106290009B4F0E94112BF0E3CF16F1E0DF0699F738
:1062A00065E2CE018F5F9B4F0E941C2BF70161912D
:1062B0007F01CE018F5F9B4F0E94112B0E151F0592
:1062C000A9F762E1CE018F5F9B4F0E941C2B88ECE7
:1062D00090E00E94EF2ACE018F5F9B4F0E94342BEB
:1062E00081EB92E00E94272B67E0CE018F5F9B4FEE
:1062F0000E941C2B65EACE018F5F9B4F0E94112BE1
:10630000CC5EDB4F0FB6F894DEBF0FBECDBFDF9182
:10631000CF911F910F91FF90EF90DF90CF90BF90A2
:10632000AF909F908F907F906F905F904F90089567
:106330001F920F920FB60F9211242F933F934F93FA
:106340005F936F937F938F939F93AF93BF93EF93DD
:10635000FF9388E293E00E940229FF91EF91BF91A1
:10636000AF919F918F917F916F915F914F913F91ED
:106370002F910F900FBE0F901F9018951F920F92A4
:106380000FB60F9211242F938F939F93EF93FF9348
:10639000E0913803F09139038081E0913E03F09160
:1063A0003F0382FD1BC09081809141038F5F8F73FB
:1063B00020914203821741F0E0914103F0E0E85D53
:1063C000FC4F958F80934103FF91EF919F918F91A7
:1063D0002F910F900FBE0F901F9018958081F4CFD2
:1063E0001F920F920FB60F9211242F933F938F930A
:1063F0009F93AF93BF938091200390912103A0912D
:106400002203B091230330911F0323E0230F2D3784
:1064100058F50196A11DB11D20931F038093200301
:1064200090932103A0932203B0932303809124032C
:1064300090912503A0912603B09127030196A11DF9
:10644000B11D8093240390932503A0932603B0935A
:106450002703BF91AF919F918F913F912F910F9003
:106460000FBE0F901F90189526E8230F0296A11DCE
:10647000B11DD2CFCF93DF93CDB7DEB72C970FB638
:10648000F894DEBF0FBECDBF789484B5826084BD22
:1064900084B5816084BD85B5826085BD85B5816028
:1064A00085BD80916E00816080936E0010928100A6
:1064B0008091810082608093810080918100816061
:1064C0008093810080918000816080938000809122
:1064D000B10084608093B1008091B00081608093AE
:1064E000B00080917A00846080937A0080917A0075
:1064F000826080937A0080917A00816080937A0034
:1065000080917A00806880937A001092C100E091B7
:106510003803F091390382E08083E0913403F091F5
:1065200035031082E0913603F091370380E18083D8
:1065300010924003E0913C03F0913D0386E080839C
:10654000E0913A03F0913B03808180618083E09188
:106550003A03F0913B03808188608083E0913A03A5
:10656000F0913B03808180688083E0913A03F09151
:106570003B0380818F7D808388E090E09E838D83C4
:1065800089E090E098878F838AE090E09A878987F6
:1065900087E090E09C878B8780EB90E09A838983EB
:1065A00088E091E09C838B8360E084E00E94112A64
:1065B00060E084E00E94E32960E085E00E94112A07
:1065C00060E085E00E94E32984EF92E00E94272B9F
:1065D000CE0101960E944B2B8C01892B91F083E018
:1065E00093E00E94272B00E010E00E949F2C0115F1
:1065F0001105D9F30E94EE288823B9F30E94000008
:10660000F4CF60E1CE0101960E941C2B82E090E065
:106610000E94EF2AF12CE12C49815A812B813C8187
:10662000429FC001439F900D529F900D112433E073
:10663000969587953A95E1F7E816F90648F46FEFD5
:10664000CE0101960E94112B8FEFE81AF80AE4CFD1
:1066500082E090E00E94EF2A63E1CE0101960E9461
:106660001C2B82E090E00E94EF2A49815A812B8105
:106670003C81429FC001439F900D529F900D112479
:1066800023E0969587952A95E1F70817190740F4B6
:106690006FEFCE0101960E94112B0F5F1F4FE5CFC8
:1066A00082E090E00E94EF2A9ECFE8E2F3E01382BE
:1066B000128288EE93E0A0E0B0E084839583A68305
:1066C000B7838EE592E09183808385EC90E0958797
:1066D000848784EC90E09787868780EC90E0918BAC
:1066E000808B81EC90E0938B828B82EC90E0958B99
:1066F000848B86EC90E0978B868B118E128E138E96
:10670000148E089597FB072E16F4009407D077FD9A
:1067100009D00E94963307FC05D03EF490958195F0
:106720009F4F0895709561957F4F0895AA1BBB1BDD
:1067300051E107C0AA1FBB1FA617B70710F0A61B81
:10674000B70B881F991F5A95A9F780959095BC01A2
:10675000CD010895EE0FFF1F0590F491E02D0994EF
:04676000F894FFCFDB
:1067640068000B001000800A00000001901414005F
:10677400000120140A000001501301000001000070
:106784000000000000000000000000000000000005
:10679400400A0000000190141400000100140A00D3
:1067A4000001990B04040101000000000000000036
:1067B40000000000000000000000400A000000018A
:1067C40090141400000100140A000001990C010344
:1067D40004010000000000000000000000000000B0
:1067E40000000000400A00000001901414000001A1
:1067F40010140A000001A0130100000100000000B1
:106804000000000000000000000000000000000084
:10681400000A0000000160141400000100140000CC
:10682400000100130A010001000000000000000044
:1068340000000000000000000000A00F0F00000591
:10684400603232000002500F0F000005000000000B
:106854000000000000000000000000000000000034
:1068640000000000500F0F000005603232000002EB
:10687400A00F0F0000050000000000000000000051
:106884000000000000000000000000000000000004
:10689400000F0F000005003232000002000F0F004D
:1068A40000050000000000000000000000000000DF
:1068B4000000000000000000000000000000242987
:1068C4008428B1287129E228C028D428652D506174
:1068D40070657220627573790D0A00652D506170C0
:1068E400657220627573792072656C656173650DDC
:1068F4000A00652D50617065722044656D6F0073E8
:10690400686F77206472617720696D6167650D0A2D
:1069140000736C6565702E2E2E007374617465208F
:10692400484947482C2072657365740073686F7713
:1069340020322D6772617920696D6167650D0A00E7
:1069440073686F7720342D6772617920696D616790
:10695400650D0A00652D506170657220696E697459
:106964000D0A00652D506170657220696E6974208E
:0A6974006661696C65640D0A00009D
:00000001FF
